:100000000C94AD070C94D5070C94D5070C94D50728
:100010000C94D5070C94D5070C94D5070C94D507F0
:100020000C94D5070C94D5070C9467190C94D61929
:100030000C94D5070C94D5070C94D5070C94D507D0
:100040000C94D5070C94D5070C94D5070C94D507C0
:100050000C94D5070C94D5070C94D5070C94081C68
:100060000C94D5070C94D5070C94D5070C94D507A0
:100070000C94D5070C94D5070C94D5070C94D50790
:100080000C94D5070C94D5070C94D5070C94D50780
:100090000C94D5070C94D5070C94D5070C94D50770
:1000A0000C94D5070C94D5070C94D50744617900BE
:1000B00041636374004C6F616E00436170616369FA
:1000C0007479200047756E732000050512151F1501
:1000D0000905082466E766244120596573202042FB
:1000E000204E6F000042726F6F6B6C796E00436F31
:1000F0006E65792049736C616E64004D616E686154
:100100007474656E0043656E7472616C2050617228
:100110006B0047686574746F0042726F6E78000000
:100120004C7564657300537065656400576565645C
:100130000041636964004865726F696E6500436FD2
:100140006361696E65002000200003081F051F1F02
:10015000151B1F11111F110E1F15111F05011F1156
:100160001D1F041F001F0010101F1F041B1F101055
:100170001F061F1F011F1F111F1F05071F311F1FF4
:10018000051B17151D011F011F101F0F100F1F0C3E
:100190001F1B041B071C071915130C121E1F120C22
:1001A0001E12120C121F0C1A14041F052E2A1E1FD9
:1001B000021C001D00201D001F041A011F001E0448
:1001C0001E1E021E1E121E3E120C0C123E1E0206A7
:1001D00014120A020F121E101E0E100E1E081E1AF6
:1001E000041A2E281E1A12161F111F001F001D159B
:1001F0001711151F07041F17151D1F151D01011FBE
:100200001F151F17151F00170000100020100000F9
:10021000030004083E09093E3F25251A1E2121122C
:100220003F21211E3F2525213F0505011E21293A99
:100230003F04043F213F21001021211F3F040A31C8
:100240003F2020203F02023F3F02043F1E21211E8B
:100250003F0909061E21112E3F09093622252519BD
:10026000013F01011F20201F0F10201F3F10103FD2
:100270003B04043B03043807312D2321102A2A3C78
:100280003F2424181C2222141824243F1C2A2A2C20
:10029000047E05014C52523E3F040438243D2000A8
:1002A0004040443D3F081422213F20003E04043ECC
:1002B0003E04023C1C22221C7E22221C1C22227E86
:1002C0003E040204242A2A12021F22201E20201E7D
:1002D0000E10201E3E10103E360808364E50503E7E
:1002E000322A26221E29251E223F200032292926B5
:1002F0001221251A0C0A3F08172525191E25251835
:10030000013905031A25251A0629291E002F000088
:10031000002000004020000000030000000000005A
:10032000003E5B4F5B3E3E6B4F6B3E1C3E7C3E1C7B
:10033000183C7E3C181C577D571C1C5E7F5E1C00C1
:10034000183C1800FFE7C3E7FF0018241800FFE778
:10035000DBE7FF30483A060E2629792926407F053B
:100360000507407F05253F5A3CE73C5A7F3E1C1C51
:1003700008081C1C3E7F14227F22145F5F005F5F11
:1003800006097F017F006689956A606060606094FD
:10039000A2FFA29408047E040810207E2010080802
:1003A0002A1C08081C2A08081E101010100C1E0C0D
:1003B0001E0C30383E3830060E3E0E06000000009F
:1003C0000000005F00000007000700147F147F1486
:1003D000242A7F2A122313086462364956205000CB
:1003E00008070300001C2241000041221C002A1CB7
:1003F0007F1C2A08083E08080080703000080808A2
:100400000808000060600020100804023E514945C1
:100410003E00427F400072494949462141494D33DF
:100420001814127F1027454545393C4A4949314146
:10043000211109073649494936464949291E000014
:100440001400000040340000000814224114141469
:100450001414004122140802015909063E415D5955
:100460004E7C1211127C7F494949363E414141225E
:100470007F4141413E7F494949417F090909013E88
:10048000414151737F0808087F00417F41002040AF
:10049000413F017F081422417F404040407F021CC1
:1004A000027F7F0408107F3E4141413E7F090909D8
:1004B000063E4151215E7F091929462649494932A4
:1004C00003017F01033F4040403F1F2040201F3F6A
:1004D0004038403F631408146303047804036159EF
:1004E000494D43007F414141020408102000414131
:1004F000417F0402010204404040404000030708DD
:100500000020545478407F284444383844444428D8
:10051000384444287F385454541800087E0902187F
:10052000A4A49C787F0804047800447D4000204007
:10053000403D007F1028440000417F40007C04784B
:1005400004787C080404783844444438FC18242493
:100550001818242418FC7C08040408485454542413
:1005600004043F44243C4040207C1C2040201C3C90
:100570004030403C44281028444C9090907C446487
:10058000544C44000836410000007700000041361A
:10059000080002010204023C2623263C1EA1A161A0
:1005A000123A4040207A38545455592155557941D2
:1005B0002154547841215554784020545579400CA9
:1005C0001E5272123955555559395454545939558A
:1005D0005454580000457C410002457D42000145CD
:1005E0007C40F0292429F0F0282528F07C5455453A
:1005F000002054547C547C0A097F493249494932CD
:100600003248484832324A4848303A4141217A3AE1
:1006100042402078009DA0A07D39444444393D40AB
:1006200040403D3C24FF2424487E4943662B2FFC58
:100630002F2BFF0929F620C0887E09032054547906
:10064000410000447D413048484A32384040227AD7
:10065000007A0A0A727D0D19317D2629292F282654
:100660002929292630484D4020380808080808085C
:100670000808382F10C8ACBA2F102834FA00007BB5
:10068000000008142A142222142A140895002200BB
:1006900095AA005500AAAA55AA55AA000000FF0075
:1006A000101010FF00141414FF001010FF00FF10B2
:1006B00010F010F0141414FC001414F700FF0000E4
:1006C000FF00FF1414F404FC141417101F10101F63
:1006D000101F1414141F00101010F0000000001F51
:1006E000101010101F10101010F010000000FF105C
:1006F0001010101010101010FF10000000FF140058
:1007000000FF00FF00001F10170000FC04F4141489
:100710001710171414F404F40000FF00F714141455
:1007200014141414F700F7141414171410101F10D5
:100730001F141414F4141010F010F000001F101FF8
:100740000000001F14000000FC140000F010F01066
:1007500010FF10FF141414FF141010101F000000DD
:1007600000F010FFFFFFFFFFF0F0F0F0F0FFFFFFE1
:100770000000000000FFFF0F0F0F0F0F3844443838
:10078000447C2A2A3E147E02020606027E027E0273
:1007900063554941633844443C04407E201E200692
:1007A000027E020299A5E7A5991C2A492A1C4C72CF
:1007B00001724C304A4D4D303048784830BC625A56
:1007C000463D3E494949007E0101017E2A2A2A2AE6
:1007D0002A44445F444440514A444040444A5140C2
:1007E0000000FF0103E080FF000008086B6B083683
:1007F00012362436060F090F0600001818000000F4
:100800001010003040FF0101001F01011E00191DE2
:100810001712003C3C3C3C0000000000D5F08D1459
:10082000A1C881CFD9F1AF2000F0F89C8E878387D3
:100830008E9CF8F00000FEFF0303030303070EFC89
:10084000F80000FEFF0303030303070EFCF800009B
:10085000FFFF00000000000000FFFF0000FEFF831C
:1008600083838383C7EE7C380000F8FC0E07030304
:1008700003070EFCF800003F7FE0C08080C0E07FEF
:100880003FFFFF01010101010101FFFF0000FFFF28
:100890000C0C0C0C1C3E77E3C100007FFFC0C0C0F5
:1008A000C0C0E0703F1F00001F3F70E0C0C0C0E04C
:1008B000703F1F00007FFFC1C1C1C1C1E3773E1C73
:1008C00000001F3F70E0C0C0C0E0703F1F0000008C
:1008D000000001FFFF010000004861726461737352
:1008E000272063617263617373212100646F6C6CF4
:1008F000617273206F6E204F666669636572007463
:1009000068656D2120596F7520666F756E642000D3
:10091000596F75206B696C6C656420616C6C206F1D
:100920006600596F75206B696C6C6564206F6E652D
:10093000212100002020596F75206D697373656453
:1009400021212100006861766520746F2072756E28
:100950002100616E792067756E732120596F7500D3
:10096000596F7520646F6E27742068617665007416
:1009700068656D2100596F752063616E277420735F
:1009800068616B6500616E20616C6C657921210086
:10099000596F75206C6F7374207468656D20696E73
:1009A00000756E697473206F663A2000596F752068
:1009B000666F756E642000323030206275636B7331
:1009C0003F006D6F726520706F636B657473206696
:1009D0006F72007472656E6368636F61742077690B
:1009E00074680057696C6C20796F75206275792086
:1009F00061206E65770057696C6C20796F75207384
:100A00006D6F6B652069743F006C696B6520676F63
:100A10006F642073747566662121006865726520B5
:100A20007468617420736D656C6C730054686572D2
:100A300065277320736F6D65207765656400646F4B
:100A40006C6C6172733F007370656369616C2066E2
:100A50006F72203430300073617475726461792074
:100A60006E69676874002E3434206D61676E756D31
:100A700020666F72006261726574746120666F72C5
:100A80000034303020646F6C6C6172733F005769C2
:100A90006C6C20796F7520627579206100616674D5
:100AA000657220796F75210064657075746965736E
:100AB0002061726500206F662068697300616E6452
:100AC00020004F66666963657220486172646173D5
:100AD0007300696E2074686520737562776179218F
:100AE00000596F752077657265206D75676765645D
:100AF00000617265206F7574726167656F7573212F
:100B000021212100636F6B65206275737421205071
:100B100072696365730050696773206D6164652055
:100B20006120626967007072696365732121210029
:100B30006174206F7574726167656F75730062759B
:100B400079696E67206865726F696E6500416464DB
:100B50006963747320617265007261696421212187
:100B6000210066726F6D206C617374207765656B10
:100B70002773006368656170206865726F696E65D0
:100B80000050696773206172652073656C6C696ED3
:100B90006700626F74746F6D6564206F75742121D6
:100BA0002100576565642070726963657320686110
:100BB0007665006C756465732121210073656C6C2A
:100BC000696E6720636865617000526976616C20A8
:100BD0006465616C6572732061726500746F646135
:100BE000792100626F72726F776564206D6F6E6538
:100BF0007900596F7520616C72656164790021001C
:100C0000596F7520646F6E27742068617665206166
:100C10006E7900004F6F707321002100596F7520AD
:100C200063616E2774206166666F726400004F6FA7
:100C30007073210021006D6F72652000596F75205F
:100C400063616E277420636172727900004F6F7068
:100C5000732100596F7527726520646561642121D5
:100C6000006265656E206869742100596F7527768A
:100C700065006D69737365642121005468657900AE
:100C8000796F752121200054686579277265206687
:100C90006972696E672061740041204669676874F3
:100CA0002020422052756E004552524F5220004182
:100CB0006D7400536176696E677300596F75206FAC
:100CC000776500596F7520686176650057697468AB
:100CD00064726177204D6F6E6579004465706F7343
:100CE0006974204D6F6E657900426F72726F772064
:100CF0004D6F6E657900506179204C6F616E000018
:100D00000051747900507269636500436F737473A6
:100D100000596F7520686176650053656C6C200022
:100D20004275792000000075703F00646F63746F36
:100D30007220746F2073657720796F7500646F6C13
:100D40006C61727320666F7220610057696C6C2051
:100D5000796F7520706179203130303000596F75AE
:100D600072206865616C74683A20007374696C6CF9
:100D700020616674657220796F7521002070696743
:100D80007300546865726520617265200042656970
:100D90006E67206368617365642121005769746818
:100DA00064726177204D6F6E6579004465706F7372
:100DB0006974204D6F6E65790042616E6B00426F01
:100DC00072726F77204D6F6E657900526570617930
:100DD000204C6F616E004C6F616E20536861726BC6
:100DE000004A65742066726F6D200053656C6C203C
:100DF0004472756773004275792044727567730099
:100E00005472656E6368636F61740042616E6B005B
:100E10004C6F616E20536861726B004A65740054B8
:100E200072656E6368636F61740053656C6C204417
:100E30007275677300427579204472756773004854
:100E40006974207468652053747265657473212118
:100E50000076312E302E3100536C616E67696E273B
:100E6000001E1E0000C08000000000000000008086
:100E70007807067880000000000000000000C040F5
:100E8000000000033CC10204081020C000FF000065
:100E90000000FF00C02010080404C2390700003819
:100EA000509090902324485060812608E70090E7F6
:100EB00008260160504826A1909090503000000014
:100EC0000000010222322A2422100A080C081221F2
:100ED000242A320203000000000000080B00020276
:100EE00002000009040000010202000005240010B5
:100EF000010524010101042402060524060001075E
:100F000005810310004009040100020A00000007E7
:100F100005020240000007058302400000040309A7
:100F20000412010002EF020140412336800001015A
:100F300002030141726475696E6F204C4C4300419D
:100F4000726475696E6F204C656F6E6172646F00BC
:100F500003051F0E0400851CC62E11241FBECFEFF3
:100F6000DAE0DEBFCDBF12E0A0E0B1E0ECE4FBE6EA
:100F700002C005900D92A236B107D9F727E0A2E68C
:100F8000B2E001C01D92AC3AB207E1F717E0CCEA3B
:100F9000D7E004C02197FE010E94A133CB3AD107CC
:100FA000C9F70E94061D0C9499350C940000E2EFDD
:100FB000F2E0A0E0B8E000800EBC8111012C119796
:100FC000A0FDFDCF0192B9F70DB40895480F592F38
:100FD000511D1416150684F5803891056CF597FFA0
:100FE00002C090E080E04138510514F040E850E044
:100FF000481BFB01E770FF2721E001C0220FEA95A3
:10100000EAF777FF02C0695F7F4FFB0133E0F59598
:10101000E7953A95E1F7F695FE2FEE27F795E795D8
:10102000E80FF91FEE50FD4F415030F08191DF0184
:101030001197822B8C93F8CF08956F927F928F92A5
:101040009F92AF92BF92CF92DF92EF92FF920F9357
:101050001F93CF93DF93DC01FA01149131965491E1
:101060003196C12FD0E0222309F1CC24C394D12C96
:10107000852F877011F4D12CC12CE52EE694E694CF
:10108000E694EC0CFD2CF11CEC9EC001ED9E900D45
:10109000FC9E900D1124033011F4880F991F289F96
:1010A0007001299FF00C1124EE0DFF1D7D01EC0E47
:1010B000FD1E1E141F040CF06BC0A038B1050CF00F
:1010C00067C0CB01850F911D181619060CF060C082
:1010D000603471050CF05CC0309709F459C0362FAC
:1010E0003770CB0177FD079623E0959587952A9574
:1010F000E1F7282F77FF04C0332311F02FEF280FDB
:10110000662777276A1B7B0BB7FD02C070E060E0A3
:1011100090E89A1B40E8E416F1040CF4912F961B1A
:10112000E22E022E000CFF08DE2CD0942F3F0CF094
:10113000D12C41E0852F877009F440E0B52EB6949C
:10114000B694B6944B0DE40EF11C89E0E816F10458
:1011500014F048E0421BB42EBD182D0D40E82403C6
:1011600070011124AE0DBF1DA60FB71F1D9D600D90
:10117000711D1124AF01460F571FC32E032E000C03
:10118000DD08033009F4C7C090F4023009F474C0DC
:10119000DF91CF911F910F91FF90EF90DF90CF9053
:1011A000BF90AF909F908F907F906F9008950A3F6F
:1011B000A1F1B20E0B3F61F72B1551F3BD016E503B
:1011C0007D4F10E000E0091708F09FC0FA01E00F22
:1011D000F11FE491F0E04F010C2C02C0880C991C27
:1011E0000A94E2F727FD06C0FB018081F82CF094F9
:1011F0008F218083332361F0273054F47B01F0E8A2
:10120000EF0EF11CA92CA094F70180818A21808324
:101210000F5F1F4F6F5F7F4FD6CFB20E2B1509F4B4
:10122000B7CFBD016E507D4F10E000E0091708F008
:1012300066C0FA01E00FF11FE491F0E04F010C2CC1
:1012400002C0880C991C0A94E2F727FD04C0FB0138
:10125000808188298083332351F0273044F47B0137
:10126000F0E8EF0EF11CF7018081892980830F5F80
:101270001F4F6F5F7F4FDACF6FEF70E0032E02C01A
:10128000660F771F0A94E2F760957095972E8B2C66
:10129000820E281509F47CCF8D010E501D4FF12CC4
:1012A000E12CE91630F5FA01EE0DFF1DE491F0E0B6
:1012B0003F010C2C02C0660C771C0A94E2F727FD54
:1012C00005C0F8018081862386298083332359F065
:1012D00027304CF45801F0E8AF0EB11CF5018081C5
:1012E000892187298083FFEFEF1AFF0A0F5F1F4FC5
:1012F000D8CF2F5F4C0F5D1FA058BF4FCACF2F5FB5
:101300004C0F5D1FA058BF4F89CF2F5F4C0F5D1F43
:10131000A058BF4F51CFE92EF12CFA01E60FF71F6D
:10132000AE50BD4F60E870E06E197F09CE19DF093D
:101330008E01000F111F41E050E07A01032E01C021
:10134000EE0C0A94EAF7592F4B2D892E932ECF934A
:10135000DF93ED01EF96EF962296A590C590992028
:1013600059F0AE9C5001CE9C600127302CF4F880DF
:10137000D094FD20FB28F99222233AF0FC90C094EF
:10138000FC20FA28FD920C94C60911965A9529F76B
:101390004A9551F0582D23951124E00FF11DA60F09
:1013A000B11DC60FD11DD9CFDF91CF911124F0CE41
:1013B0000F9302E020E00E941D080F9108952F92E4
:1013C0003F924F925F926F927F928F929F92AF92D5
:1013D000BF92CF92DF92EF92FF920F931F93CF9322
:1013E000DF93CDB7DEB728970FB6F894DEBF0FBEF8
:1013F000CDBF6F836A0119011C830B83FE82ED82CE
:10140000811128C005E010E029E030E03A8329830B
:10141000B6010D2C000C880B990B0E9405304B0176
:101420005C015F8151111DC0E0E6F7E090E080E0D3
:1014300018861F828C159D050CF02BC124813581E7
:101440004F8158854217530714F438872F8301962C
:101450003696F0CF04E010E048E050E05A8349832C
:10146000D7CF20E030E040E05FE30E9464304B01E2
:101470005C0120E030E0A9010E943F3320E030E031
:1014800040E05FE387FD30C0C501B4010E94D33165
:101490000E94B13278876F83A6018F819885481B9F
:1014A000590BE0E6F7E090E080E0B12CA12C2F8111
:1014B000388582179307ECF086E0829FF001839FC6
:1014C000F00D1124E05AF84F90E080E0D12CC12CAF
:1014D00084179507BCF424813581C216D3060CF419
:1014E000690101963696F4CFC501B4010E94D2314C
:1014F000CFCF24813581A216B3060CF45901019691
:101500003696D5CFB801110F880B990B0E94053084
:101510002B013C01B5016C0D7D1D072E000C880BC5
:10152000990B0E94053020E030E040EE5FE30E941E
:10153000D3316B017C0120E030E040E05FE3C30188
:10154000B2010E9464309B01AC01C701B6010E9448
:1015500064306B017C0120E030E0A9010E943F3340
:1015600020E030E040E05FE387FD89C0C701B601BD
:101570000E94D3310E94B13202E410E0061B170B27
:10158000F10111830083B501BB0C880B990B0E94FC
:10159000053020E030E040EE5FE30E94D331A3014C
:1015A00092010E9464304B015C0120E030E0A9010F
:1015B0000E943F3320E030E040E05FE387FD64C0FD
:1015C000C501B4010E94D3310E94B132600F711F76
:1015D000EB81FC817183608329813A81B901330FEA
:1015E000880B990B0E94053020E030E040E05FE37B
:1015F0000E9464306B017C014F815885BA01550F00
:10160000880B990B0E9405309B01AC01C701B60104
:101610000E9464306B017C0120E030E0A9010E944F
:101620003F3320E030E040E05FE387FD85C0C70145
:10163000B6010E94D3310E94B1322AE230E0C901E2
:10164000861B970BED81FE819183808328960FB6D0
:10165000F894DEBF0FBECDBFDF91CF911F910F91E8
:10166000FF90EF90DF90CF90BF90AF909F908F90C2
:101670007F906F905F904F903F902F900895C7019B
:10168000B6010E94D23176CFC501B4010E94D23199
:101690009BCFB801110F880B990B0E94053020E0F9
:1016A00030E040E05FE30E9464302B013C01EF81B9
:1016B000F885BF01FF0F880B990B0E9405309B0135
:1016C000AC01C301B2010E9464302B013C0120E057
:1016D00030E0A9010E943F3320E030E040E05FE3CA
:1016E00087FD25C0C301B2010E94D3310E94B132EF
:1016F00022E430E0C901861B970BF10191838083BE
:101700008FEF9FEFEB81FC819183808329813A8168
:10171000B901330F880B990B0E94053020E030E0AF
:1017200040E05FE30E946430A501940171CFC301E2
:10173000B2010E94D231DACFC701B6010E94D23184
:101740007ACFFC018091F102882311F13FB7F89420
:1017500082E08093E9002091F200822F90E0181639
:10176000190614F481E090E0882339F0289844E6C3
:101770004093F0024091F1004083222339F0209100
:10178000F200211103C02BE62093E8003FBF08952B
:101790008FEF9FEF08952FB7F89483E08093E900CF
:1017A0009091E800892F807295FF04C09091F2001B
:1017B00080E4891B2FBF08958091E80281110DC03C
:1017C00082E08093E40284E08093E5021092E702D5
:1017D0001092E60281E08093E80284EE92E00895A0
:1017E000CF93DF931F92CDB7DEB76983DC01ED9114
:1017F000FC910280F381E02D41E050E0BE016F5F7B
:101800007F4F09950F90DF91CF91089583E08093EA
:10181000E9008091F200882319F08AE38093E800C0
:1018200008950E94CB0B90E00895CF93DF931F9211
:10183000CDB7DEB7FC018485958597FD08C02FEFF5
:101840003FEF358724870F90DF91CF910895CE0128
:1018500001960E94A10B019719F4898190E0F3CFC2
:101860008FEF9FEFF0CF0F931F93CF93DF931F92D4
:10187000CDB7DEB78C01FC018485958597FF0BC041
:10188000CE0101960E94A10B019771F4898190E02D
:10189000F80195878487F801848595850F90DF91FD
:1018A000CF911F910F9108958FEF9FEFF1CFFC0122
:1018B0008485958597FD0BC09FB7F89482E080934F
:1018C000E9008091F2009FBF90E0019608959FB7D4
:1018D000F89482E08093E9008091F2009FBF90E04D
:1018E00008954091DE025091DF022091DC02309198
:1018F000DD0242175307B4F49091E8009570E1F3CC
:101900009091E80092FD19C08093F1008091DE0271
:101910009091DF0201968F739927892B19F48EEF2E
:101920008093E8008091DE029091DF02019690930F
:10193000DF028093DE0281E0089580E00895DF9267
:10194000EF92FF920F931F93CF93DF93D82E8A01CC
:10195000EB017B01E40EF51ECE15DF0559F0D7FE35
:1019600012C0FE0184910E94710C21968111F4CF66
:101970000FEF1FEFC801DF91CF911F910F91FF90E3
:10198000EF90DF9008958881EECF0F931F93CF9350
:10199000DF931F92CDB7DEB782E0898342E450E047
:1019A0006BED7EE080E80E949F0C0E94DC0BDC0166
:1019B00012960D911C910115110589F0D801ED9138
:1019C000FC910280F381E02DBE016F5F7F4FC80163
:1019D000099597FD04C0F80100851185ECCF898138
:1019E0000F90DF91CF911F910F910895615030F0CA
:1019F0002091F100FC0120830196F8CF289884E61D
:101A00008093F00208953FB7F8948091D8029091A6
:101A1000D902A091DA02B091DB0226B5A89B05C0DD
:101A20002F3F19F00196A11DB11D3FBFBA2FA92F5D
:101A3000982F8827BC01CD01620F711D811D911D5A
:101A400042E0660F771F881F991F4A95D1F70895C6
:101A50008F929F92AF92BF92CF92DF92EF92FF92BE
:101A60006B017C010E94030D4B015C01C114D10488
:101A7000E104F104B9F00E94030D681979098A099B
:101A80009B09683E73408105910580F321E0C21AED
:101A9000D108E108F10888EE880E83E0981EA11CA9
:101AA000B11CE4CFFF90EF90DF90CF90BF90AF904C
:101AB0009F908F9008958F929F92AF92BF92CF92F6
:101AC000DF92EF92FF920F931F93CF93DF936C01FE
:101AD0007B018A0180910C01882309F45CC080910C
:101AE000F102882309F457C08091E30280FF05C00A
:101AF0008091E00082608093E000E801B12C8AEFE1
:101B0000A82E93E0892E2AE3922E209711F4BB2071
:101B1000D9F10E94CB0B81110AC0AA94AA20D9F155
:101B200061E070E080E090E00E94280DEECF8C171D
:101B30001D0611F00CF08C2F9FB7F8948092E900ED
:101B40002091E80025FD02C09FBFDFCF282F30E0A5
:101B5000C21BD30BF701815020F041914093F1005B
:101B6000FACFE20EF31EBB2021F09092E800B12CD8
:101B7000EBCF8091E80085FDE7CF9092E800BB2491
:101B8000B394209709F3F3CF5D9884E68093E20243
:101B9000101611063CF081E090E0F60193838283F9
:101BA00010E000E0C801DF91CF911F910F91FF90ED
:101BB000EF90DF90CF90BF90AF909F908F9008955F
:101BC0000895DB0114964D915C9115976D917C9170
:101BD000DC01ED91FC910280F381E02D09942F92BC
:101BE0003F924F925F926F927F928F929F92AF92AD
:101BF000BF92CF92DF92EF92FF920F931F93CF93FA
:101C0000DF9300D000D000D0CDB7DEB7782E662E9F
:101C10005A0128E0422E512C811103C099E0492E2F
:101C2000512CCE0101967C018E010D5F1F4F9E014C
:101C30002B5F3F4FA501662D872D0E94DF09B5015F
:101C40000B2C000C880B990B0E94053020E030E033
:101C500040E05FE30E9464306B017C0120E030E0F3
:101C6000A9010E943F3320E030E040E05FE387FDC0
:101C700024C0C701B6010E94D3310E94B1328B014A
:101C800080E6C82E87E0D82E049D1001059D300CFB
:101C9000149D300C1124F12CE12C912C812C8A14F0
:101CA0009B04B4F589819A81662019F0801691060B
:101CB0004CF42D818E0D9F1D0BC0C701B6010E94F3
:101CC000D231DBCF2B81A70142195309840F951F15
:101CD0007720A1F02093950720939407809396078F
:101CE000B60180E997E00E94E10D9FEF891A990AF9
:101CF00086E0C80ED11CE40CF51CD1CF20939F07C1
:101D000020939E078093A007B6018AE997E0EBCF66
:101D100026960FB6F894DEBF0FBECDBFDF91CF91F0
:101D20001F910F91FF90EF90DF90CF90BF90AF90F9
:101D30009F908F907F906F905F904F903F902F90EB
:101D40000895EF92FF920F931F93CF93DF938C012F
:101D50007B01D0E0C0E0F701EC0FFD1F649166232A
:101D600061F0D801ED91FC910190F081E02DC80166
:101D70000995892B11F02196EECFCE01DF91CF91FD
:101D80001F910F91FF90EF900895AF92BF92CF9265
:101D9000DF92EF92FF920F931F93CF93DF936C012B
:101DA0007B018B01040F151FEB015E01AE18BF080C
:101DB000C017D10759F06991D601ED91FC910190BE
:101DC000F081E02DC6010995892B79F7C501DF91D6
:101DD000CF911F910F91FF90EF90DF90CF90BF9028
:101DE000AF9008952D9A0895BC0190E080E00C9486
:101DF000280D8FB18095807F669B88601C9B8460D6
:101E0000089581EC80937C0085B1806F85B984B1A1
:101E1000877E84B984B1876E84B95E9A5F988AB1EF
:101E2000806D8AB9769A6E9881B3806F81BB8998EC
:101E300080B38D7080BB80E58CBD81E08DBD85E079
:101E400090E00E94F40E5F9A85E090E00E94F40E0C
:101E50005E985C98ECE1F8E084918EBD00000DB4D2
:101E600007FEFDCF319688E0E932F807A9F75C9AC2
:101E700081E88093640080916500816080936500B3
:101E8000089590916A02982329F490916B02982307
:101E900081E009F480E00895CF93C82F0E94F90EE5
:101EA000982F9C2381E09C1380E0CF91089580E0DF
:101EB0000C94D70780389105B8F460347105A0F40C
:101EC00020E191E061FD94E060FD990F62FD929543
:101ED000687F269FD0011124A80FAE50BD4F8C9172
:101EE00040FF03C0892B8C93089590958923FBCFE5
:101EF0002F923F924F925F926F927F928F929F921A
:101F0000AF92BF92CF92DF92EF92FF920F931F9307
:101F1000CF93DF937C016B0188248394912CD0E0D4
:101F2000C0E005E010E096EF692E77247A942CEF5C
:101F3000A22EBB24BA94842F8470582E842F8270D2
:101F4000482E842F8870382E4170242E219682E0EE
:101F5000880E911CA80CB91C552091F041E0B801E5
:101F60006C0D7D1DC7018C0F9D1F0E945A0F41E013
:101F7000B6016C0F7D1FC8018E0D9F1D0E945A0F68
:101F8000442091F041E0B601601B710BC7018C0F3A
:101F90009D1F0E945A0F41E0B6016C1B7D0BC801CA
:101FA0008E0D9F1D0E945A0F332091F041E0B60123
:101FB0006C0F7D1FC701801B910B0E945A0F41E0DF
:101FC000B8016C0D7D1DC7018C1B9D0B0E945A0F23
:101FD000222091F041E0B6016C1B7D0BC701801BF4
:101FE000910B0E945A0F41E0B601601B710BC701B3
:101FF0008C1B9D0B0E945A0FC017D10754F4B7FCDD
:10200000A5CF0150110982E0680E711CA60CB71C07
:102010009DCFDF91CF911F910F91FF90EF90DF90B7
:10202000CF90BF90AF909F908F907F906F905F9078
:102030004F903F902F9008952F923F924F925F9232
:102040006F927F928F929F92AF92BF92CF92DF92C8
:10205000EF92FF920F931F93CF93DF93EC0141E038
:102060006FE370E00E945A0F41E065E370E0CE013B
:102070000E945A0F41E06AE370E0CE0105960E948B
:102080005A0F41E06AE370E0CE0105970E945A0FB3
:1020900022242394312CF12CE12C05E010E036EFC2
:1020A000432E55245A944CEFC42EDD24DA948FEF3E
:1020B000E81AF80A82E0280E311CC20CD31C470132
:1020C0008C0E9D1E41E058018AE3A80EB11CB5019B
:1020D000C4010E945A0F3E016E187F0841E0B5010D
:1020E000C3010E945A0F41E08AE3A82EB12CA01A26
:1020F000B10AB501C4010E945A0F41E0B501C30104
:102100000E945A0F47018AE3880E911C41E0B401F6
:102110005E01A00EB11EC5010E945A0F41E0B4013C
:102120003E01601A710AC3010E945A0F9AE3892E78
:10213000912C8E189F0841E0B401C5010E945A0FEE
:1021400041E0B401C3010E945A0FE016F1069CF071
:10215000DF91CF911F910F91FF90EF90DF90CF9083
:10216000BF90AF909F908F907F906F905F904F90B7
:102170003F902F900895D7FC9ACF0150110982E02B
:10218000480E511CC40CD51C92CF8F929F92AF92D7
:10219000BF92CF92DF92EF92FF920F931F93CF9354
:1021A000DF936D3089F0C0906802D09069026A3088
:1021B000D1F4109267021092660288E0C80ED11C1A
:1021C000D0926902C092680281E090E0DF91CF91E5
:1021D0001F910F91FF90EF90DF90CF90BF90AF9045
:1021E0009F908F9008950091660210916702E5E03C
:1021F0006E9FE0011124C45EDC4F4801F12CF5E034
:10220000E12CFF1629F0CE010196FE01E490EC01CD
:10221000B12CA12C4E2D4170B6016A0D7B1DC4015D
:102220000E945A0FE694FFEFAF1ABF0A88E0A81683
:10223000B10481F7F394EFEF8E1A9E0AF6E0FF12D5
:10224000DECF0A5F1F4F1093670200936602BCCF78
:10225000DF92EF92FF920F931F93CF93DF937C0156
:10226000D22E8B01040F111DEB0177FF02C0D0E0CD
:10227000C0E0C8010134110514F080E490E0C817F3
:10228000D9073CF44D2DBE01C7010E945A0F21967B
:10229000F0CFDF91CF911F910F91FF90EF90DF90E2
:1022A00008952F923F924F925F926F927F928F92FA
:1022B0009F92AF92BF92CF92DF92EF92FF920F93D5
:1022C0001F93CF93DF9300D000D000D0CDB7DEB7FF
:1022D0006C01762E542E4901602E98E0A92EB12C67
:1022E000611103C089E0A82EB12CCE0101967C01BA
:1022F0008E010D5F1F4F9E012B5F3F4FA401652D87
:10230000872D0E94DF0909811A81552011F1B4013E
:10231000990C880B990B0E94053020E030E040E0DA
:102320005FE30E9464301B012C0120E030E0A90132
:102330000E943F3320E030E040E05FE387FD0CC0C7
:10234000C201B1010E94D3310E94B132C616D70634
:1023500044F48D809E8009C0C201B1010E94D23137
:10236000F3CF8B809C80C61AD70ACA9CB001CB9C45
:10237000700DDA9C700D1124060F171FC40104970D
:102380006620B1F061E070E0711002C062E070E0C0
:10239000060F171F6C01C6012FEFC21AD20AC8140C
:1023A000D90491F020E045E0B8010E942811F3CF54
:1023B00061E070E0711002C062E070E0600F711FB8
:1023C00040E55FE00E94D80926960FB6F894DEBF7C
:1023D0000FBECDBFDF91CF911F910F91FF90EF9076
:1023E000DF90CF90BF90AF909F908F907F906F9035
:1023F0005F904F903F902F9008950F93CF93DF936E
:10240000EC019E816A3059F48D818C836985960F29
:102410009E8381E090E0DF91CF910F910895262F68
:1024200061E0690F2A3398F4203378F5273249F1B7
:1024300040F4213261F198859C5F8C81890F8C83F7
:10244000E8CF2C3231F12E32B1F72FE309C021341D
:1024500090F32B35C0F08FE9820F27548A3158F75B
:10246000062E000C770B8C81082E000C990B3F81F7
:102470000AEF313009F00BEF42E152E00E941D08F3
:10248000DACF21E4EDCF2154EBCF2C5FE9CF2EE35F
:10249000E7CF20E4E5CF0F93CF93DF93EC019E814C
:1024A0006A3059F48D818C836985960F9E8381E013
:1024B00090E0DF91CF910F910895262F61E0690F91
:1024C0002A3398F4203378F5273249F140F4213249
:1024D00061F198859D5F8C81890F8C83E8CF2C32C8
:1024E00031F12E32B1F72FE309C0213490F32B35AF
:1024F000C0F08FE9820F27548A3158F7062E000C5E
:10250000770B8C81082E000C990B3F810AEF31303C
:1025100009F00BEF4AE451E00E941D08DACF21E4F4
:10252000EDCF2154EBCF2C5FE9CF2EE3E7CF20E4B2
:10253000E5CFEEEAF2E086EC92E030E020E0419177
:10254000519161917191240F351F8E179F07B9F733
:1025500080917B0290917C02821B930B0895CF9314
:10256000C82F84E00E94410F811107C0CC2381F065
:1025700088E00E94410F882359F01092D202809186
:102580008D0290918E029093CF028093CE0281E0D3
:10259000CF910895E0E9F7E08AE48583848387E3B7
:1025A000868368ED70E0CF010E94A10E8BE490E07D
:1025B0000E941C1087E690E00C941C10CF92DF92D2
:1025C000EF92FF920F931F93CF93DF9346E770E054
:1025D00060E085E090E00E94E60746E76FE370E088
:1025E00085E090E00E94E60721E046E365E070E0C8
:1025F00090E080E00E94281121E046E365E070E071
:102600008FE790E00E94281141E065E070E085E0EE
:1026100090E00E94780F42E065E070E08AE790E089
:102620000E94780F44E06AE370E08AE790E00E943D
:10263000780F48E06AE370E085E090E00E94780F50
:1026400080918F02C2E4D7E0811122C00AE010E03D
:10265000F12CE12C8AE0C82ED12C8091900290912F
:102660009102E816F90684F58FEFE81AF80AD0927D
:102670006702C09266021093690200936802BE016D
:1026800084EA97E00E94E10D065F1F4F2696E5CF92
:102690001AE0F12CE12C0AE08091900290919102D5
:1026A000E816F9068CF400939F0700939E07109399
:1026B000A007BE018AE997E00E94E10D8FEFE81ABA
:1026C000F80A175F2696E8CFDF91CF911F910F91FF
:1026D000FF90EF90DF90CF900895BC01EAE9F7E01A
:1026E00096E0958394838CE08683CF010C94E10D72
:1026F00090E080E008958F929F92AF92BF92EF9208
:10270000FF920F931F93CF93DF93CDB7DEB7A197BF
:102710000FB6F894DEBF0FBECDBF7C01FA01CB012E
:1027200019A2223008F42AE08E010F5D1F4F822E7D
:10273000912CB12CA12CBF01A50194010E94A131C3
:10274000F901CA016A3074F5605DD8016E938D019C
:10275000232B242B252B79F790E080E0109789F02C
:10276000FD0101900020E9F73197AF014A1B5B0B97
:10277000D701ED91FC910280F381E02DB801C701F2
:102780000995A1960FB6F894DEBF0FBECDBFDF91BD
:10279000CF911F910F91FF90EF90BF90AF909F90BE
:1027A0008F900895695CD1CFCF92DF92EF92FF9224
:1027B0000F931F93CF93DF9377FF21C06A017B01B3
:1027C000EC01E881F9810190F081E02D6DE209953D
:1027D0008C0144275527BA014C195D096E097F0900
:1027E0002AE0CE010E947B13800F911FDF91CF91D1
:1027F0001F910F91FF90EF90DF90CF9008952AE006
:10280000DF91CF911F910F91FF90EF90DF90CF90CC
:102810000C947B13CF93DF93CFE1D0E020E04AE02C
:1028200067E170E0CE010E9428112196CF36D105D4
:10283000A9F783E280939F0780939E0788E18093A6
:10284000A0074091770250917802609179027091CF
:102850007A028AE997E0DF91CF910C94D413BC01FE
:10286000EAE9F7E09AE09583948388E18683CF01D3
:102870000E94E10D48E566E170E08EE190E00E9483
:10288000E60748E561E270E08EE190E00E94E6072D
:1028900021E04CE066E170E08EE190E00E942811BA
:1028A00021E04CE066E170E085E790E00E942811AD
:1028B0000E940A1441ED50E068E170E08FE690E07C
:1028C0000C94D809CF92DF92EF92FF920F931F934F
:1028D000CF93C82F8B0169017A016E5F7F4F4AEC5D
:1028E00050E00E94D809CA5FEAE9F7E0C583C483D3
:1028F0000683B701A601CF01CF911F910F91FF90E1
:10290000EF90DF90CF900C94D413CF93DF9380910E
:10291000CE029091CF024197029768F5C8E2D0E0CD
:1029200020E047E065E270E0CE010E942811219688
:10293000CF37D105A9F7E0918B02F0918C02EE0F11
:10294000FF1FEE0FFF1FEA56FD4F208131814281AC
:102950005381609177027091780280917902909111
:102960007A020E9491339B01AC0165E270E088E23B
:1029700090E00E946214DF91CF910C940A14CF93DF
:10298000DF93EC0188819981009711F00E94433414
:10299000198218821D821C821B821A82DF91CF91BC
:1029A0000895FC0180819181009711F00C944334CB
:1029B0000895CF93C82F8091CC029091CD020196BB
:1029C0009093CD028093CC02109276020E94352F14
:1029D00021EE3EE240E050E00E9438316058714CF8
:1029E0008F4F9F4F60939602709397028093980247
:1029F000909399020E94352F29E53BE140E050E099
:102A00000E94383168577C4E8F4F9F4F60939A02D7
:102A100070939B0280939C0290939D020E94352F9D
:102A200023E230E040E050E00E9438319B01AC01ED
:102A3000265F3F4F4F4F5F4FA4E6B0E00E945731F3
:102A400060939E0270939F028093A0029093A102D4
:102A50000E94352F2BE230E040E050E00E943831F8
:102A60009B01AC012F5D3F4F4F4F5F4FAAE0B0E09D
:102A70000E9457316093A2027093A3028093A40234
:102A80009093A5020E94352F20E130E040E050E015
:102A90000E9438319B01AC01295F3F4F4F4F5F4F80
:102AA000AAE0B0E00E9457316093A6027093A7029B
:102AB0008093A8029093A9020E94352F25E030E070
:102AC00040E050E00E9438319B01AC012F5F3F4F46
:102AD0004F4F5F4FAAE0B0E00E9457316093AA02C7
:102AE0007093AB028093AC029093AD02CC23C1F102
:102AF0006091830270918402809185029091860298
:102B00000E9405302DEC3CEC4CE85FE30E94643001
:102B10000E94E7320E94B132609383027093840274
:102B2000809385029093860260917F02709180026B
:102B300080918102909182020E94053024E13EEA58
:102B400047E85FE30E9464300E94E7320E94B1329E
:102B500060937F027093800280938102909382023F
:102B60001092D202CF9108950C9422310F931F93AB
:102B7000CF93DF938C01EB01FC0180819181009761
:102B8000E1F06881798161157105A9F04281538175
:102B90002C813D814217530770F00E9492358C8141
:102BA0009D81F801958384831D821C82DF91CF91E2
:102BB0001F910F9108950E94433488819981F801F3
:102BC000918380838A819B81938382838C819D8181
:102BD00095838483198218821B821A82E5CF0F9312
:102BE0001F93CF93DF93EC0188819981009759F06F
:102BF0002A813B812617370730F081E0DF91CF91A2
:102C00001F910F9108958B016F5F7F4F0E94CC340D
:102C1000009759F0998388831B830A832C813D8117
:102C2000232B59F7FC011082E8CF80E0E7CFEF9229
:102C3000FF920F931F93CF93DF93EC017B01CB01A6
:102C40000E94942F0097A9F00C811D81080F191F75
:102C5000B801CE010E94EF15882361F028813981E7
:102C60008C819D81B701820F931F0E948D2F1D8340
:102C70000C8381E0DF91CF911F910F91FF90EF9036
:102C80000895EF92FF920F931F93CF93DF93FB0171
:102C9000E080F180E114F10441F480E0DF91CF9114
:102CA0001F910F91FF90EF900895048115810115F8
:102CB0001105B1F0EC018C819D81080F191FB8013D
:102CC000CE010E94EF15882341F3288139818C8140
:102CD0009D81B701820F931F0E9492351D830C8343
:102CE00081E0DCCFEF92FF920F931F93CF93DF939E
:102CF000EC018B016115710551F0CB010E94942FFD
:102D00007C01BC01CE010E94EF1581110BC0CE01E8
:102D10000E94BF14CE01DF91CF911F910F91FF90C0
:102D2000EF900895FD82EC82B801888199810E941C
:102D30008D2FF0CFFC011182108213821282158236
:102D400014820C947216CF93DF93EC0162307105FC
:102D500001F148F46115710581F061307105B1F040
:102D60006FE171E00CC064307105C9F0A8F0653006
:102D70007105B1F760E271E002C06EE371E0CE016F
:102D80000E949A16CE01DF91CF91089566E371E01B
:102D9000F6CF61E371E0F3CF6CE271E0F0CF66E271
:102DA00071E0EDCFCF93DF93EC016230710501F15B
:102DB00048F46115710581F061307105B1F064EE80
:102DC00070E00CC064307105C9F0A8F06530710581
:102DD000B1F765EE70E002C069E171E0CE010E94DA
:102DE0009A16CE01DF91CF91089562E171E0F6CF9E
:102DF00065E071E0F3CF6BEF70E0F0CF6EEE70E066
:102E0000EDCFEF92FF920F931F93CF93DF93EC01DF
:102E10007B018A01BA010E94EF1581110BC0CE011E
:102E20000E94BF14CE01DF91CF911F910F91FF90AF
:102E3000EF9008951D830C83B701888199810E94CA
:102E40009235F0CFFB0101900020E9F73197AF01F7
:102E5000461B570B0C9401170F931F93CF93DF93CF
:102E6000CDB7DEB762970FB6F894DEBF0FBECDBF09
:102E70008C01CB01F801118210821382128215821B
:102E800014824AE0BE016F5F7F4F0E949D2FBE01FA
:102E90006F5F7F4FC8010E94221762960FB6F894A9
:102EA000DEBF0FBECDBFDF91CF911F910F9108956F
:102EB0000F931F93CF93DF93CDB7DEB7A2970FB6D3
:102EC000F894DEBF0FBECDBF8C01CB01BA01F80173
:102ED0001182108213821282158214822AE0AE01BE
:102EE0004F5F5F4F0E94A82FBE016F5F7F4FC801E9
:102EF0000E942217A2960FB6F894DEBF0FBECDBF78
:102F0000DF91CF911F910F9108952F923F924F9291
:102F10005F926F927F928F929F92AF92BF92CF9269
:102F2000DF92EF92FF920F931F93CF93DF93CDB772
:102F3000DEB762970FB6F894DEBF0FBECDBF2C018F
:102F40009E012F5F3F4F490139011C01D12CC12C3B
:102F500010E000E0B12CA12CF1014191519161915F
:102F600071911F01CE010D960E945817E988FA88C9
:102F7000CE010D960E94D114B601CE010D960E948D
:102F8000A31689899A89E80EF91EFFEFEF1AFF0A46
:102F9000F301E192F1923F01CE010D960E94D1140E
:102FA000F3E0CF16D1040CF03FC0AE14BF040CF414
:102FB00057012FEFC21AD20A36E0C316D10461F6C8
:102FC00080E6C82E87E0D82EF12CE12C150183E095
:102FD000E816F1040CF01801B701CE010D960E941D
:102FE000A316BE01635F7F4FC6010E94B615CE01D6
:102FF0000D960E94D11468E471E0C6010E94171674
:10300000712C612CF401808191819101281B390B75
:103010006216730674F466E471E0C6010E94171626
:103020003FEF631A730AEECF0E151F0514F68701E2
:10303000C0CFF20141915191619171912F01CE0167
:103040000D960E945817BE01635F7F4FC6010E9414
:103050004116CE010D960E94D114FFEFEF1AFF0A20
:1030600026E0C20ED11C32E0830E911C86E0E816E9
:10307000F10409F0ABCFF092CB02E092CA0281E0FA
:103080008093C8020A0D1B1D073111050CF480E066
:103090008093C90262960FB6F894DEBF0FBECDBF13
:1030A000DF91CF911F910F91FF90EF90DF90CF9024
:1030B000BF90AF909F908F907F906F905F904F9058
:1030C0003F902F900895EF92FF920F931F93CF930D
:1030D000DF9300D000D000D0CDB7DEB78091CE0214
:1030E0009091CF02099709F05EC00E9499128C015D
:1030F000BC01CE0101960E942C17ED80FE80CE010E
:1031000001960E94D11481E08093950780939407E3
:103110001092960764EC70E080E997E00E94A10E9F
:1031200040917D0250917E02052E000C660B770BBC
:1031300080E997E00E94D41387E190E08E199F09FF
:10314000880F991F880F991F809395078093940784
:10315000109296076AEB70E080E997E00E94A10E5A
:10316000A801110F660B770B80E997E00E94D4133A
:1031700010E000E021E041E068E070E0C8010E945A
:1031800028110F5F1F4F00381105A1F726960FB6C3
:10319000F894DEBF0FBECDBFDF91CF911F910F918D
:1031A000FF90EF90089540918702509188026091BE
:1031B000890270918A02CE0101960E945817ED8013
:1031C000FE80CE0101960E94D11400E210E00E199B
:1031D0001F09000F111F000F111F8091CE02909147
:1031E000CF029C01255031092230310508F052C030
:1031F00021E020939507209394071092960760EBA7
:1032000070E0059711F465EB70E080E997E00E94AB
:10321000A10E4AEC50E061E070E083E190E00E9492
:10322000D80989E1809395078093940710929607B7
:103230008091CE029091CF02059719F540918302BB
:1032400050918402609185027091860280E997E036
:103250000E94D4134AEC50E061E070E0C801069788
:103260000E94D8090093950700939407109296073F
:1032700040918702509188026091890270918A0280
:1032800073CF40917F0250918002609181027091D2
:103290008202DCCF81E0809395078093940710929F
:1032A00096076CEA70E080E997E00E94A10E8EE03C
:1032B0008093950780939407109296074091CC02D3
:1032C0005091CD02052E000C660B770BBFCF1F92DD
:1032D0000F920FB60F9211248F939F938091E1006C
:1032E0009091E100937F9093E10083FF0FC01092D3
:1032F000E90091E09093EB001092EC0092E3909340
:10330000ED001092F10298E09093F00082FF22C04D
:1033100093E09093E9009091F200992319F09AE3D9
:103320009093E8009091E202992341F09091E2029B
:1033300091509093E202911101C05D9A9091F00238
:10334000992341F09091F00291509093F0029111E5
:1033500001C0289A84FF18C08091E2008E7E8160AF
:103360008093E2008091E1008F7E8093E100809164
:10337000E3028E7E80618093E3029F918F910F9094
:103380000FBE0F901F90189580FFF7CF8091E2003D
:103390008E7E80618093E2008091E1008E7E80933A
:1033A000E1008091E3028E7E8160E5CF1F920F9253
:1033B0000FB60F921124CF92DF92EF92FF920F93EC
:1033C0001F932F933F934F935F936F937F938F93AD
:1033D0009F93AF93BF93EF93FF93CF93DF93CDB7BB
:1033E000DEB76C97DEBFCDBF1092E9008091E80098
:1033F00083FF25C068E0CE0145960E94F60C82EF5F
:103400008093E8008D8987FF39C09091E80090FF94
:10341000FCCF982F907609F034C19E894F89588D42
:103420002F89F88C911131C0803861F58091E102CB
:103430008093F1001092F1008EEF8093E8006C967B
:103440000FB6F894DEBF0FBECDBFDF91CF91FF91D5
:10345000EF91BF91AF919F918F917F916F915F910C
:103460004F913F912F911F910F91FF90EF90DF901F
:10347000CF900F900FBE0F901F9018959EEF9093D6
:10348000E800C7CF1092F100D5CF913059F48111E7
:10349000D3CF4130510581F68091E1028D7F809339
:1034A000E102CACF933049F48111C6CF41305105B2
:1034B00019F68091E1028260F2CF953041F480915B
:1034C000E80080FFFCCF20682093E300B5CF963062
:1034D00009F0A9C00B8D1C8D22E01092E90010921A
:1034E000DF021092DE02F2122EC01092DD02109264
:1034F000DC020E94C50C1F8299E09983FA8291E058
:103500009E8390EA98879AEF99872091DE02309106
:10351000DF02275F3F4F3C832B838D831092E900AE
:103520001092DF021092DE021093DD020093DC02A3
:1035300049E050E0BE016F5F7F4F80E00E949F0C2A
:103540000E94C50C79CF1093DD020093DC020E942B
:10355000DC0BDC0112960D911C910115110509F48B
:1035600051C1D801ED91FC910480F581E02DBE019F
:103570006B5E7F4FC8010995009709F03EC1F801C5
:1035800000851185EACFF3E0FF120EC08F898823F2
:1035900009F440C0823061F440E860E18FE39FE0CD
:1035A0000E94521C811148CF81E28093EB0047CFEB
:1035B000813029F440E86BE083E39FE0F1CF833072
:1035C00099F70E94DC0BDC011296ED90FC908E01C5
:1035D0000F5F1F4F6801E114F10479F0D701ED91FD
:1035E000FC910680F781E02DB801C7010995080F0D
:1035F000111DF701E084F184EECFD8011C92F60191
:1036000001900020E9F73197BF016C197D0940E076
:10361000C601C6CF6DE17FE0FB01449150E080E838
:103620000E949F0C09CF973009F4BECF983021F447
:1036300081E08093F10000CF993009F0FDCE8370D6
:1036400009F0B2CFE8E1F1E081E031E096E32191C9
:10365000222371F08093E9003093EB00DF01119792
:103660002C912093EC009093ED008F5F873079F7D9
:103670008EE78093EA001092EA008F898093F1022E
:10368000DBCE8B8D9C8D1092E9001092DF021092A0
:10369000DE029093DD028093DC02898D811192C05D
:1036A0008E899D89913A49F4813209F07DCF47E0B6
:1036B00050E065E071E080E0B3CF913209F074CF63
:1036C000833269F48F89988DB0E0A0E08093010186
:1036D00090930201A0930301B0930401ADCE803218
:1036E00069F48091E80082FFFCCF67E085E091E01B
:1036F0000E94F60C8BEF8093E8009ECE823209F098
:103700009BCE8F8980930C01EEEFFFE7859194911A
:103710008B3F9C4D51F1E0E0F8E0809105019091E4
:103720000601A0910701B0910801803B9440A105DA
:10373000B105F1F480910C0180FD1AC0EE3F8AE0E2
:10374000F80789F587E797E7918380838091600088
:103750008093E00288E19BE00FB6F894A8958093EF
:1037600060000FBE9093600067CEEEEFFAE0D5CF19
:10377000808191818737974709F05ECEA895809127
:1037800060008861809360008091E0028093600017
:10379000EE3F2AE0F20789F08091FE0A9091FF0A3D
:1037A0009183808349CE808191818737980751F238
:1037B0009093FF0A8093FE0AC5CF1092FF0A1092E1
:1037C000FE0A3ACE0E94DC0BDC0112960D911C9190
:1037D0000115110509F4E8CED801ED91FC91019095
:1037E000F081E02DBE016B5E7F4FC801099581110C
:1037F00023CEF80100851185EBCF181619060CF4BD
:103800001BCED2CEF1E0FF12BECE61E27FE004CF4C
:103810001F920F920FB60F9211242F933F938F9305
:103820009F93AF93BF938091D4029091D502A091C2
:10383000D602B091D7023091D30223E0230F2D3767
:1038400058F50196A11DB11D2093D3028093D40297
:103850009093D502A093D602B093D7028091D8025C
:103860009091D902A091DA02B091DB020196A11DDC
:10387000B11D8093D8029093D902A093DA02B0933D
:10388000DB02BF91AF919F918F913F912F910F904C
:103890000FBE0F901F90189526E8230F0296A11DCA
:1038A000B11DD2CFEF92FF920F931F93CF93DF936F
:1038B000F82E192FE62E042F81E0860F880F0E9424
:1038C000710C83E00E94710CCF2DD12FEC0EFD2ED8
:1038D000F11CCE15DF05B9F007FF13C0FE0184917E
:1038E0000E94710C182F80E00E94710C8123219698
:1038F0008111EFCFDF91CF911F910F91FF90EF904A
:1039000008958881EDCF81E0F5CFCF93DF931092BA
:10391000F5061092F40688EE93E0A0E0B0E0809304
:10392000F6069093F706A093F806B093F90682E2A4
:1039300091E09093F3068093F2068FEF9FEF9093C0
:10394000FF068093FE061092A7071092A6078CE44C
:1039500091E09093A5078093A40710929D07109281
:103960009C0780E491E090939B0780939A0798E0EE
:103970009093A30781E08093A20710929F07109273
:10398000A00710929E078093A107109293071092B0
:10399000920724E331E030939107209390079093AE
:1039A00099078093980710929507109296071092A6
:1039B000940780939707C0E6D7E0198218821B828C
:1039C0001A821D821C8250E040E06AEF71E0CE0155
:1039D0000E940117269687E0C039D80771F7C2E424
:1039E000D7E0198218821B821A821D821C8250E045
:1039F00040E06AEF71E0CE010E940117269687E051
:103A0000C036D80771F7DF91CF910895CF93DF9338
:103A1000CDB7DEB760970FB6F894DEBF0FBECDBF4F
:103A2000789484B5826084BD84B5816084BD85B599
:103A3000826085BD85B5816085BD80916E008160A5
:103A400080936E001092810080918100826080934B
:103A5000810080918100816080938100809180004D
:103A600081608093800080919100826080939100BA
:103A7000809191008160809391008091900081609D
:103A8000809390008091C10084608093C1008091F8
:103A9000C10082608093C1008091C10081608093E9
:103AA000C1008091C30081608093C3008091C000F9
:103AB00082608093C0008091C20081608093C200C8
:103AC00080917A00846080937A0080917A0082608D
:103AD00080937A0080917A00816080937A0080914F
:103AE0007A00806880937A001092F1021092E102CD
:103AF0001092E3028091D70081608093D70080EA22
:103B00008093D80089B5806189BD89B5826089BDFF
:103B100009B400FEFDCF61E070E080E090E00E941B
:103B2000280D8091D8008F7C80618093D80080918F
:103B3000E000807F8093E0008091E1008E7E8093A2
:103B4000E1008DE08093E200559A209A0E94010FD7
:103B500082E480930001809164008E7F80936400F2
:103B600080917A00806480937A0080917A0086FD4B
:103B7000FCCF00917800109179000E94030DAB01F9
:103B8000BC01C801B0E0A0E0DC01992788276C01E6
:103B90007D01C40ED51EE61EF71EC701B601209199
:103BA0006400216020936400611571058105910511
:103BB00011F00E94842F1092CF021092CE02109228
:103BC000D2020E94010F0E94570F80E80E944C0F02
:103BD0008823A9F05C9885EA8EBD00000DB407FE2D
:103BE000FDCF5C9A2E982F982D988091640080626A
:103BF0008093640081E083BF889513BEFCCF84E08E
:103C00000E944C0F882309F448C02D9884E80E9434
:103C10004C0F8823E1F00E94F20E88EC90E00E94A5
:103C2000F40E2F9882E090E00E9422318F3F29F01D
:103C30006FEF82E090E00E942A3184EF91E00E94D1
:103C4000F40E2F9A84E80E944C0F8111FBCF84E17F
:103C50000E944C0F8823E1F00E94F20E88EC90E065
:103C60000E94F40E2E9882E090E00E942231882378
:103C700029F060E082E090E00E942A3184EF91E038
:103C80000E94F40E2E9A84E10E944C0F8111FBCF0A
:103C900088EC90E00E94F40EB2CF0E94F20E82E017
:103CA00090E00E94B415882309F441C03E9A3F9ADF
:103CB00081E090E00E94B41581FF13C0082F0470CA
:103CC000302E82FD2E9801EF1FEFB8E0AB2EB12C05
:103CD00080E40E944C0F882369F12E9A2F9A0E944B
:103CE000F20E82E390E00E94F40E0E94F90E811120
:103CF000F8CFE2E04E2E512C612C712C8FB7F89446
:103D00004091D4025091D5026091D6027091D702B1
:103D10008FBF80916402882309F4D0C0109264029E
:103D200080E090E0892B51F30E940000E7CF3E989D
:103D30003F98BECF332029F00430110511F42E9A9C
:103D40002F9881E00E94D707980117FF04C022270F
:103D50003327201B310B27703327C80117FD079627
:103D6000A3E095958795AA95E1F717FF05C0019700
:103D7000A501421B530B9A01BC017695762F66274D
:103D8000779567956E507D4FF12CE12C2501421AF5
:103D9000530A8E3F5FEF950709F43EC0DB0150E008
:103DA00040E0F701E75DF74F4F013B01F0E86F0E90
:103DB000711C8F3F980781F0F401E40FF51FE49127
:103DC000022E01C0EE0F0A94EAF75496FC91549724
:103DD000EF2B5496EC93549721153105B9F0F4016B
:103DE000E40FF51F24906301C40ED51EE22DF0E010
:103DF000042C02C0F595E7950A94E2F7FE87ED875B
:103E0000F6012488FD852F2AF601248A4F5F5F4F33
:103E100011964835510569F60196F8E5EF0EF11C4B
:103E200060587F4F40EBE416F10409F0B2CF0E94D6
:103E3000570F8FE090E00E94F40E0F5F1F4F093183
:103E4000110509F045CF332011F02F9A2D9880E904
:103E500091E00E94F40E0E94F20E81E090E00E9438
:103E6000B41580FF3ECF8AE090E00E94B4159FEF2A
:103E7000980F9E3F08F035CF22E330E03093670281
:103E80002093660228E330E03093690220936802B1
:103E90000BE010E0682F84EA97E00E94C510C8018B
:103EA0000E94B4150F5F1F4F0131110599F70E9451
:103EB000570F88EE93E00E94F40E13CF80916502B5
:103EC000942F981B892F90910001891748F48F5FD8
:103ED000891708F025CF81E083BF889513BE20CFD6
:103EE00081E0809364024093650280916202909128
:103EF00063020196909363028093620280916B0249
:103F000080936A020E94F90E80936B028091D20224
:103F10008111F5C02091CE023091CF02E2EFF2E0A4
:103F200081118FEF00248193819381938193039476
:103F3000D1F71092690210926802109267021092F3
:103F400066021092D1021092D0022130310561F444
:103F50008091CC029091CD024F9734F087E190E0B0
:103F60009093CF028093CE028091CE029091CF02A7
:103F70008831910508F0AEC4FC01EF53F04E0C946B
:103F8000A133D91F1D20EC20C720C7206821912113
:103F9000AA210F22A8209A229A229A229A22A622A5
:103FA000D2226F22F122F12294239423942394238A
:103FB000012441E65EE070E060E090E080E00E9475
:103FC000D80941E65EE070E060E082E690E00E94A1
:103FD000D8098AE290E090936702809366028FE0AE
:103FE00090E0909369028093680268E57EE084EA3D
:103FF00097E00E94A10E87E680939507809394072F
:104000008AE38093960761E57EE080E997E00E946D
:10401000A10E6FE37EE080E697E00E94721681E0D9
:1040200090E09093CB028093CA021092C902109242
:10403000C80241E050E060E04DC00E94631860910A
:10404000C6027091C702CE0101960E94D216CE011F
:1040500001960E946D13CE0101960E94D11465E372
:104060007EE080E697E00E9472166AE27EE086E6D5
:1040700097E00E9472166FE17EE08CE697E00E9466
:1040800072166BE17EE082E797E00E9472168091E3
:10409000C6029091C702892B09F057C060E17EE00B
:1040A00088E797E00E9472166BE07EE08EE797E06B
:1040B0000E94721686E090E09093CB028093CA0231
:1040C0001092C90281E08093C8024091CA025091C7
:1040D000CB0261E080E00E94EF0D2091CA02309196
:1040E000CB0200E04091C8026091C9028091D002E9
:1040F0009091D1020E94511181E08093D202C09030
:10410000CE02D090CF02B8E1CB16D10408F07CC427
:10411000F601E357FF4D0C94A133872487248724AD
:104120008724872487248724632BD72AD72AD72A52
:10413000DB2ADB2ADB2AD72AD72ADB2A592C592C5F
:10414000592C592C592C592CD72A84E090E0B4CF03
:104150000E94631860E07EE0CE0101960E949A16EC
:10416000CE0101960E946D13CE0101960E94D114DA
:104170008EEA92E00E9485174091CA025091CB02CC
:104180006091C8028091C9020E94EF0DB5CF0E94D4
:1041900063188091CE029091CF0266EF7DE0039785
:1041A00011F06BEE7DE0CE0101960E949A16CE01D1
:1041B00001960E946D13CE0101960E94D11486E9EA
:1041C00092E00E9485174091CA025091CB02609103
:1041D000C8028091C9027FCF0E94631861EE7DE022
:1041E000CE0107960E949A166091C6027091C7028E
:1041F000CE0101960E94D216BE016F5F7F4FCE01A5
:1042000007960E944116CE0101960E94D1141A828F
:1042100019821C821B821E821D826F817885611526
:10422000710531F04B855C85CE0101960E94011726
:10423000CE0101960E946D13CE0101960E94D11409
:1042400070E6E72E77E0F72E70E060E08B010F5FFD
:104250001F4F8091C6029091C702681779070CF032
:10426000B801CE0101960E94D216BE016F5F7F4F4A
:10427000C7010E94B615CE0101960E94D114A6E096
:10428000EA0EF11CB8010530110501F71093CB02BD
:104290000093CA0281E08093C9028093C80245E07E
:1042A00050E061E00E94EF0D2091CA023091CB02F4
:1042B00000E04091C8026091C9028091D0029091C3
:1042C000D1020E945111CE0107960E94D11414CF41
:1042D0000E94631866ED7DE0CE0101960E949A1659
:1042E000CE0101960E946D13CE0101960E94D11459
:1042F0006BEC7DE080E697E00E9472166EEB7DE04D
:1043000086E697E00E94721682E090E09093CB02DE
:104310008093CA021092C9021092C80242E050E093
:104320008ACE0E94631869EB7DE0CE0101960E945F
:104330009A16CE0101960E946D13CE0101960E943D
:10434000D1146BEA7DE080E697E00E9472166CE97A
:104350007DE0D6CF6DE87DE082E497E00E947216A2
:1043600062E87DE088E497E00E9472166091940212
:1043700070919502CE0101960E942C17BE016F5FCD
:104380007F4F88E497E00E944116CE0101960E947B
:10439000D1146CE77DE088E497E00E9417166BE685
:1043A0007DE08EE497E00E9472166DE57DE084E585
:1043B00097E00E9472166091920270919302CE0172
:1043C00001960E942C17BE016F5F7F4F84E597E036
:1043D0000E944116CE0101960E94D11484E090E023
:1043E000909391028093900210928F020E94DE12AD
:1043F00082E4809395078093940787E380939607E0
:1044000069E97CE080E997E00E94A10E83E490E0F6
:104410000E941C1087E690E00E941C106DCE0E9446
:10442000352F6B017C0167E87CE082E497E00E9415
:10443000721660E87CE088E497E00E94721687E0DC
:1044400090E090938E0280938D0283E090E09093B1
:1044500091028093900210928F02C701B601A301CE
:1044600092010E943831672B79F46BE77CE088E495
:1044700097E00E94171662E77CE08EE497E00E94C6
:1044800072160E94DE1238CE6BE67CE088E497E07C
:104490000E94171661E67CE08EE497E00E94721697
:1044A000809192029091930203979093930280934C
:1044B0009202181619062CF363E57CE084E597E078
:1044C0000E94721684E090E0909391028093900293
:1044D00087E190E090938E0280938D02D2CF6BE4BF
:1044E0007DE082E497E00E9472166DE37DE088E44F
:1044F00097E00E9472166BE27DE08EE497E00E94E6
:10450000721667E27DE084E597E00E94721684E00F
:1045100090E0909391028093900210928F020E94FB
:10452000DE120E94CA1281E090E090938E02809386
:104530008D02E2CD0E94DE128091CE029091CF02D8
:104540000A9709F4D9CD0E94CA12D6CD64E571E06C
:1045500082E497E00E9422176BE671E088E497E01E
:104560000E94221760E871E08EE497E00E94221713
:1045700067E971E084E597E00E9422176EEA71E036
:104580008AE597E00E94221785E090E090939102DF
:104590008093900281E080938F020E94DE128FE070
:1045A00090E0C3CF6AEF71E082E497E00E942217A7
:1045B00062EC71E088E497E00E94221761ED71E0FF
:1045C0008EE497E00E94221783E090E0909391029E
:1045D0008093900210928F020E94DE1287E190E099
:1045E000A4CF60E27DE0419711F06AE17DE082E4D2
:1045F00097E00E94721660918B0270918C02CE013E
:1046000001960E94A316BE016F5F7F4F82E497E080
:104610000E944116CE0101960E94D11466E27DE00F
:1046200088E497E00E94721665E27DE08EE497E0F0
:104630000E9472168091CE029091CF026BE07DE0D5
:10464000419711F065E07DE084E597E00E947216E5
:1046500061E17DE08AE597E00E94721685E090E0D6
:10466000909391028093900281E080938F020E9448
:10467000DE12E0918B02F0918C02EE0FFF1FEE0F25
:10468000FF1FEA56FD4F20813181428153816091A5
:10469000460770914707E5E0E69FC001E79F900D50
:1046A00011246AE070E00F960E9462148091CE029D
:1046B0009091CF024197E9F42091870230918802CE
:1046C0004091890250918A026EE270E087E390E0A7
:1046D0000E9462140E94851461E07DE0CE01019683
:1046E0000E949A16CE0101960E942F14CE010196C7
:1046F000ECCD87E380939F0780939E078EE28093A3
:10470000A007E0918B02F0918C02EE0FFF1FEE0FDD
:10471000FF1FE255FD4F40815181628173818AE91B
:1047200097E00E94D413D6CF66EF7CE083319105E9
:1047300059F069EE7CE08431910531F06BED7CE05D
:10474000459711F06CEC7CE082E497E00E947216D1
:1047500060E07DE088E497E00E9472166FEF7CE0F5
:104760008EE497E00E94721680918D0290918E02E5
:104770006BEB7CE0059711F063EB7CE084E597E060
:104780000E94721663EC7CE08AE597E00E94721644
:1047900085E090E0909391028093900281E0809375
:1047A0008F020E94DE1280918D0290918E020597F9
:1047B000F9F4209183023091840240918502509156
:1047C000860265E270E082E390E00E94621420912C
:1047D0008702309188024091890250918A026EE2EC
:1047E00070E087E390E00E9462146FEA7CE076CF8D
:1047F00020917F023091800240918102509182028B
:10480000E0CF60917F02709180028091810290914F
:1048100082020091870210918802209189023091D2
:104820008A02600F711F821F931F009183021091F3
:1048300084022091850230918602601B710B820BED
:10484000930B0E94053020E030E04CEF51E40E94D1
:104850003F320E944A330E94E7320E94B1326B011C
:104860006AEF71E082E497E00E9422176FED71E039
:1048700088E497E00E9422176CEE71E08EE497E0E6
:104880000E942217B6016536710514F064E670E0E7
:10489000CE0101960E942C17BE016F5F7F4F8EE400
:1048A00097E00E944116CE0101960E94D1146BEF51
:1048B00071E084E597E00E94221710928F0284E055
:1048C00090E0909391028093900210928E02109249
:1048D0008D02D7CD85E090E09093670280936602C9
:1048E000909369028093680268EA7CE084EA97E02A
:1048F0000E94A10E4091CE025091CF02052E000CD5
:10490000660B770B84EA97E00E94D413F5CB80E81E
:104910000E94410F81111AC080E10E94410F811154
:1049200015C080E20E94410F811110C080E40E94F6
:10493000410F81110BC088E00E94410F811106C018
:1049400084E00E94410F882309F45EC0A090CA024F
:10495000B090CB023090C802E090D002F090D1022B
:1049600001E09501432D6091C902C7010E945111D8
:10497000B5010B2C000C880B990B0E94053020E030
:1049800030E040E05FE30E9464306D877E878F8770
:10499000988B20E030E0A9010E943F3320E030E016
:1049A00040E05FE387FD33C06D857E858F85988904
:1049B0000E94D3310E94B1328B0188248394912CC0
:1049C000E616F7061CF032E0832E912C80E10E945F
:1049D000410F882359F1EFEFEE1AFE0AEA14FB04A7
:1049E000ECF4F092D102E092D0022091CA02309110
:1049F000CB0200E04091C8026091C9028091D002D0
:104A00009091D1020E9451110E94570F89C96D8562
:104A10007E858F8598890E94D231CCCFF1E0AF1A84
:104A2000B108B092D102A092D002DFCF80E80E94FC
:104A3000410F882371F001E0E01AF108F092D102F1
:104A4000E092D002F7FED1CF1092D1021092D002A4
:104A5000CCCF80E40E94410F8823D9F03320A9F005
:104A60008A94892891F4E00EF11EF092D102E0922E
:104A7000D0028091D0029091D1028A159B050CF44E
:104A8000B4CF41E0A41AB108CCCF3FEFE31AF30A48
:104A9000ECCF80E20E94410F8823B9F0332089F0E7
:104AA00052E08516910469F4E01AF10AF092D102FD
:104AB000E092D0028091D0029091D10297FF95CFE1
:104AC000C3CF81E0E81AF108F1CF88E00E94410FDE
:104AD000882309F459C51092D20293E0C916D10473
:104AE00009F4BFC308F05AC0B1E0CB16D10409F4F1
:104AF00086C0E2E0CE16D10409F4B0C0EF2809F078
:104B000074CF81E090E09093CF028093CE0220EDAD
:104B100037E040E050E020938702309388024093D2
:104B2000890250938A0288E893E1A0E0B0E0809384
:104B3000830290938402A0938502B0938602109220
:104B40007F021092800210928102109282021092D3
:104B5000C7021092C60210927E0210927D0284E675
:104B600090E090937C0280937B0282E390E09093AC
:104B7000930280939202EEEAF2E086EC92E01192C8
:104B80001192119211928E179F07C9F71092CD02C0
:104B90001092CC0280E00E94D91427CFF5E0CF1606
:104BA000D10409F47EC408F423C416E0C116D1046C
:104BB00009F0A4CF86E090E090938E0280938D025E
:104BC00010927702109278021092790210927A0273
:104BD000E114F10409F4C9C4EA94EF2809F005CFFF
:104BE00086E190E09093CF028093CE0280917F0285
:104BF00090918002A0918102B091820221C4D09252
:104C00008E02C0928D0292E0E916F104F1F074F484
:104C1000E114F104B9F084E090E0EA94EF2809F09F
:104C2000E4CE9093CF028093CE02DFCEE4E0EE1686
:104C3000F10489F06CF086E090E005E0E016F10404
:104C400081F3D3CE83E090E0ECCF89E090E0E9CF30
:104C500082E090E0E6CF85E090E0E3CF8091C6026D
:104C60009091C702E816F9061CF01FEFE11AF10A4D
:104C7000F092C702E092C60281E00E94D9140E941D
:104C8000352F24E130E040E050E00E9438319B01B4
:104C900041E050E050938E0240938D0210928F02BB
:104CA000FB013197E131F10508F0D6C2E65AF94D22
:104CB0000C94A1336B269226B126E426E4260F2716
:104CC0000F273C27832783278327E527E5273928D4
:104CD0005A288928F9286AEC7BE082E497E00E9450
:104CE00072166CEB7BE088E497E00E94721663EB2F
:104CF0007BE08EE497E00E94721683E090E0909350
:104D000091028093900222E030E040E050E0209356
:104D1000AA023093AB024093AC025093AD028AE0FA
:104D200090E07FCF62EA7BE082E497E00E94721617
:104D300062E97BE088E497E00E94721682E090E0EE
:104D400090939102809390028AE790E0A0E0B0E017
:104D50008093A2029093A302A093A402B093A50211
:104D6000DECF61E87BE082E497E00E94721663E7A1
:104D70007BE088E497E00E94721662E67BE08EE4B6
:104D800097E00E94721669E57BE084E597E00E9457
:104D9000721684E090E090939102809390020E94BA
:104DA000352F2EE734E040E050E00E9438316E5A53
:104DB0007C4F8F4F9F4F60939A0270939B0280931A
:104DC0009C0290939D02ABCF6DE47BE082E497E080
:104DD0000E9472166EE37BE088E497E00E947216F0
:104DE00060E37BE08EE497E00E94721666E27BE06F
:104DF00084E597E00E94721684E090E0909391021F
:104E0000809390020E94352F29EA31E640E050E07D
:104E10000E943831605B794B8F4F9F4FCCCF66E15A
:104E20007BE082E497E00E94721664E07BE088E415
:104E300097E00E94721661EF7AE08EE497E00E949C
:104E4000721683E090E090939102809390020E940A
:104E5000352F21E63AEE40E050E00E9438316058AC
:104E6000774C8E4F9F4F609396027093970280937A
:104E700098029093990253CF61EE7AE082E497E032
:104E80000E94721662ED7AE088E497E00E94721642
:104E900082E090E09093910280939002609187026B
:104EA000709188028091890290918A020E94053057
:104EB00020E030E040E450E40E943F326B017C018E
:104EC00020E030E0A9010E943F3320E030E040E0E4
:104ED0005FE387FD13C0C701B6010E94D3310E9472
:104EE000B132660F771F881F991F609387027093F6
:104EF00088028093890290938A0211CFC701B6017C
:104F00000E94D231ECCFEEEAF2E046EC52E090E0C3
:104F100080E0C190D190E190F1908C0D9D1D4E17D5
:104F20005F07B9F7C2970CF43FC382E090E02930E5
:104F3000310539F084E090E02A30310511F085E048
:104F400090E0909395028093940262EC7AE082E480
:104F500097E00E9472166DEB7AE088E497E00E9479
:104F60007216609194027091950261507109CE01A0
:104F700001960E942C17BE016F5F7F4F88E497E077
:104F80000E944116CE0101960E94D11465EB7AE091
:104F900088E497E00E94171668EA7AE08EE497E0CA
:104FA0000E9472166DE97AE084E597E00E9472161D
:104FB00084E090E0909391028093900287E090E0EB
:104FC00090938E0280938D02AACE80918702909159
:104FD0008802A0918902B0918A02843F9140A10584
:104FE000B1050CF4E1C20E94991205970CF4DCC2E1
:104FF0000E94352F23E030E040E050E00E9438313D
:105000006B016EE87AE082E497E00E947216F2E0AB
:10501000CF16D104C8F465E77AE0CD2811F066E632
:105020007AE088E497E00E94721661E87AE08EE404
:1050300097E00E94721683E090E090939102809333
:1050400090028BE090E0EDCD67E57AE088E497E0B0
:105050000E94721667E47AE08EE497E00E9472166E
:105060006EE37AE084E597E00E94721684E090E0B7
:10507000E4CF6CE27AE082E497E00E9472166BE182
:105080007AE088E497E00E94721669E07AE08EE4A4
:1050900097E00E94721666EF79E084E597E00E943F
:1050A000721684E090E090939102809390028DE0DC
:1050B00090E0B7CD8091870290918802A0918902FB
:1050C000B0918A028C329140A105B1050CF46CC2FA
:1050D00063EE79E082E497E00E94721663ED79E076
:1050E00088E497E00E94721662EC79E08EE497E023
:1050F0000E94721667EB79E084E597E00E947216D1
:1051000084E090E090939102809390028CE090E094
:1051100088CD0E94991208970CF446C20E94352F40
:1051200027E030E040E050E00E9438318B010F5F13
:105130001F4F0E94352F26E030E040E050E00E94F3
:1051400038316B01FB01EE0FFF1FEE0FFF1FE25521
:10515000FD4FA801012E000C660B770B8081918119
:10516000A281B381840F951FA61FB71F80839183EF
:10517000A283B3836CEA79E082E497E00E9472161E
:10518000B801CE0101960E942C17BE016F5F7F4FC0
:1051900082E497E00E944116CE0101960E94D1144C
:1051A00061EA79E088E497E00E947216B601CE01C8
:1051B00001960E94A316BE016F5F7F4F88E497E0BF
:1051C0000E944116CE0101960E94D11469E072E05E
:1051D0008EE497E00E9422176BE172E084E597E08D
:1051E0000E94221784E090E09093910280939002B5
:1051F00096CD69E272E082E497E00E94221768E3AC
:1052000072E088E497E00E9422176AE472E08EE47C
:1052100097E00E94221769E572E084E597E00E941A
:10522000221784E090E090939102809390020E9474
:10523000352F27E232E040E050E00E9438316650DE
:105240007F4F8F4F9F4F60939E0270939F0280937A
:10525000A0029093A10263CD5093CF024093CE025F
:10526000C4CB0E9499128C01D0928E02C0928D0202
:10527000F0928C02E0928B0218161906F4F16DE49C
:105280007CE082E497E00E9472166CE47CE088E4A3
:1052900097E00E9472166CE37CE08EE497E00E9437
:1052A000721666E37CE084E597E00E9472166091D6
:1052B0008B0270918C02CE0101960E94A316BE0152
:1052C0006F5F7F4F84E597E00E944116CE01019603
:1052D0000E94D11464E37CE084E597E00E941716F5
:1052E00084E090E0909391028093900210928F025C
:1052F0008091CE029091CF0263CEF701EE0FFF1F97
:10530000EE0FFF1FEA56FD4FC080D180E280F38090
:1053100060918702709188028091890290918A023F
:105320006C157D058E059F0544F56EE27CE082E4F8
:1053300097E00E9472166DE27CE088E497E00E949C
:1053400072166CE17CE08EE497E00E947216609128
:105350008B0270918C02CE0101960E94A316BE01B1
:105360006F5F7F4F84E597E00E94B615CE010196EE
:105370000E94D1146AE17CE0AFCF21E130E03093AC
:10538000CF022093CE0210927702109278021092F0
:10539000790210927A020E9405304B015C01C7012C
:1053A000B6010E9405309B01AC01C501B4010E9409
:1053B0003F320E94E7320E94B13260936C027093D8
:1053C0006D0280936E0290936F02012E000C220BEF
:1053D000330B06171707280739070CF006CB009385
:1053E0006C0210936D0220936E0230936F02FDCA1F
:1053F00084E090E090938E0280938D02F0928C0274
:10540000E0928B02F701EE0FFF1FEE0FFF1FE25538
:10541000FD4F80819181A281B381181619061A0669
:105420001B06BCF422E130E03093CF022093CE0281
:1054300010927702109278021092790210927A02FA
:1054400080936C0290936D02A0936E02B0936F02F2
:10545000CCCA64E17CE082E497E00E94721663E1CA
:105460007CE088E497E00E94721660E07CE08EE4C5
:1054700097E00E94721660918B0270918C02CE01AF
:1054800001960E94A316BE016F5F7F4F84E597E0EF
:105490000E94B615CE0101960E94D1146EEF7BE0FA
:1054A0001BCFD0928E02C0928D0210927702109282
:1054B00078021092790210927A02E114F10419F143
:1054C000EA94EF2809F091CA809176028823D1F1FD
:1054D00062EF7BE082E497E00E94721663EE7BE06D
:1054E00088E497E00E9472166CED7BE08EE497E012
:1054F0000E94721683E090E0909391028093900254
:1055000010928F020CCC83E190E09093CF028093B5
:10551000CE02409187025091880260918902709179
:105520008A028091830290918402A0918502B091B9
:105530008602481759076A077B070CF081CFDB0109
:10554000CA017ECF84E190E09093CF028093CE0297
:1055500028E833E140E050E020936C0230936D0284
:1055600040936E0250936F0240CA85E190E09093A1
:10557000CF028093CE028091870290918802A09101
:105580008902B0918A025CCF84E00E94410F882397
:1055900009F42BCA42E0C41AD10855E0C516D1045B
:1055A00008F023CA1092D20281E090E03ACB81E069
:1055B0000E94AF1229CA80E00E94AF12811124CA52
:1055C00088E00E94410F882309F41ECA1092D2027B
:1055D0008091CE029091CF028C30910509F44EC09B
:1055E00060F50B9709F010CA80917D0290917E02C0
:1055F000019690937E0280937D0280918702909124
:105600008802A0918902B0918A0280599140A10933
:10561000B1098093870290938802A0938902B09386
:105620008A0280917B0290917C02059790937C0284
:1056300080937B0281E090E041C08D309105E1F1E3
:10564000409709F0E1C98091870290918802A0916A
:105650008902B0918A02885E9340A109B1098093C2
:10566000870290938802A0938902B0938A0282E312
:1056700090E09093930280939202DCCF80917B0222
:1056800090917C020A9690937C0280937B02809199
:10569000870290918802A0918902B0918A02885C69
:1056A0009109A109B1098093870290938802A09380
:1056B0008902B0938A02BECF8EE090E09093CF0231
:1056C0008093CE02A1C984E00E94410F882309F48F
:1056D00040C01092D2020E94352FA30192010E9475
:1056E0003831672B682B692BB9F460E979E082E4E3
:1056F00097E00E94721665E879E088E497E00E94DE
:10570000721682E090E09093910280939002109242
:105710008F0281E090E016C065E779E082E497E0CF
:105720000E9472166FE679E088E497E00E94721694
:1057300082E090E0909391028093900210928F0209
:1057400088E090E090938E0280938D028AE090E052
:10575000B5CF88E00E94410F882309F455C9109203
:10576000D20280917D0290917E02892BE9F460E65D
:1057700079E082E497E00E94721662E579E088E4BD
:1057800097E00E94721665E479E08EE497E00E944B
:10579000721683E090E090939102809390021092B1
:1057A0008F0287E090E0CECF0E94352FA3019201B7
:1057B0000E943831672B682B692B49F464E479E047
:1057C00082E497E00E94721664E379E0ADCF8091A5
:1057D0009402909195020197909395028093940280
:1057E000181619064CF463E379E082E497E00E940E
:1057F000721662E279E098CF0E94352F23EE34E0F2
:1058000040E050E00E9438318B0102511D4F60E1B1
:1058100079E082E497E00E9472166FEF78E088E406
:1058200097E00E947216B801CE0101960E942C17D3
:10583000BE016F5F7F4F88E497E00E944116CE0162
:1058400001960E94D1146CEE78E08EE497E00E94FD
:10585000721669ED78E084E597E00E94721684E0A4
:1058600090E0909391028093900281E080938F0268
:10587000012E000C220B330B80918702909188023D
:10588000A0918902B0918A02800F911FA21FB31FBD
:105890008093870290938802A0938902B0938A0232
:1058A000803B9440A105B1050CF433CF80E190E03A
:1058B00049CF80E00E94AF128111A6C888E00E9403
:1058C000410F882309F439C18091CE029091CF0213
:1058D0008331910509F4B7C068F48131910509F469
:1058E00079C04297C1F11092D20280918D029091BD
:1058F0008E02E4CE8531910509F402C108F4CCC0D2
:10590000469789F740917702509178026091790229
:1059100070917A0280917F0290918002A091810221
:10592000B0918202841B950BA60BB70B80937F026C
:1059300090938002A0938102B093820280918702AB
:1059400090918802A0918902B0918A02840F951FDC
:10595000A61FB71F36C080918B0290918C022091B8
:105960007702309178024091790250917A02880F43
:10597000991F880F991FFC01E255FD4FC080D1800F
:10598000E280F380C21AD30AE40AF50AC082D18207
:10599000E282F3828A569D4FDC016D917D918D915B
:1059A0009C910E949133009187021091880220916E
:1059B000890230918A02DC01CB01800F911FA21F66
:1059C000B31F8093870290938802A0938902B093BB
:1059D0008A0289CF80918B0290918C02209177026C
:1059E000309178024091790250917A02880F991F84
:1059F000880F991FFC01E255FD4FC080D180E280E5
:105A0000F380C20ED31EE41EF51EC082D182E28254
:105A1000F3828A569D4FFC0160817181828193815E
:105A20000E9491330091870210918802209189028F
:105A300030918A0268017901C61AD70AE80AF90A80
:105A4000D701C601BECF4091770250917802609194
:105A5000790270917A028091830290918402A091E0
:105A60008502B0918602841B950BA60BB70B809321
:105A7000830290938402A0938502B0938602809162
:105A8000870290918802A0918902B0918A02841BBA
:105A9000950BA60BB70B95CF4091770250917802EA
:105AA0006091790270917A028091830290918402D0
:105AB000A0918502B0918602840F951FA61FB71F83
:105AC0008093830290938402A0938502B093860210
:105AD0008091870290918802A0918902B0918A02F8
:105AE000840F951FA61FB71F80938702909388028B
:105AF000A0938902B0938A0281E080937602F3CE6C
:105B000040917702509178026091790270917A0207
:105B100080917F0290918002A0918102B0918202D7
:105B2000840F951FA61FB71F80937F02909380025A
:105B3000A0938102B0938202A2CF8FB7F894C09055
:105B4000D402D090D502E090D602F090D7028FBF59
:105B50008091CE029091CF02419701E010E0029730
:105B600010F00AE010E08091720290917302A0910F
:105B70007402B0917502B701A601481B590B6A0B5C
:105B80007B0B8091700290917102823091050CF034
:105B9000F5C0453F51406105710510F40C94042592
:105BA0000196909371028093700280E80E944C0FDE
:105BB0008823C1F1C0927202D0927302E092740203
:105BC000F092750280916C0290916D02A0916E022C
:105BD000B0916F02012E000C220B330B4091770223
:105BE000509178026091790270917A026C017D0186
:105BF000C01AD10AE20AF30AC416D506E606F70669
:105C00000CF447C0040F151F261F371F009377029F
:105C1000109378022093790230937A020E948514BF
:105C20000C94042580E40E944C0F882309F443C09F
:105C3000C0927202D0927302E0927402F0927502E6
:105C400040916C0250916D0260916E0270916F02F2
:105C50002AE0209FC001219F900D1124092E000CE5
:105C6000AA0BBB0B00917702109178022091790268
:105C700030917A026A017B01C81AD90AEA0AFB0A42
:105C8000C016D106E206F3066CF0800F911FA21F2A
:105C9000B31F8093770290937802A0937902B09318
:105CA0007A02BCCF409377025093780260937902D6
:105CB00070937A02B3CF80E10E944C0F882339F1B0
:105CC000C0927202D0927302E0927402F092750256
:105CD000012E000C220B330B8091770290917802F9
:105CE000A0917902B0917A0280179107A207B307B9
:105CF0002CF0801B910BA20BB30BCBCF1092770231
:105D0000109278021092790210927A0287CF80E284
:105D10000E944C0F882321F1C0927202D09273022C
:105D2000E0927402F09275028AE0809FA001819F48
:105D3000500D1124052E000C660B770B8091770215
:105D400090917802A0917902B0917A028417950718
:105D5000A607B7079CF2841B950BA60BB70B99CF30
:105D600010927202109273021092740210927502D5
:105D700010927102109270020C9404254536510560
:105D80006105710508F011CF0C940425CF93DF93C2
:105D90008AE597E00E94D11484E597E00E94D1142F
:105DA0008EE497E00E94D11488E497E00E94D11419
:105DB00082E497E00E94D114C0E9D7E02697CE0193
:105DC0000E94D11487E0C036D807C1F7DF91CF9188
:105DD00008958F929F92AF92BF92CF92DF92EF92EF
:105DE000FF92CF93DF93EC01688179818A819B8157
:105DF000611571058105910521F464E279ED8BE56A
:105E000097E02DE133EF41E050E00E943831490145
:105E10005A019B01AC01A7EAB1E40E9457316B0122
:105E20007C01ACEEB4EFA50194010E946531C60E71
:105E3000D71EE81EF91EF7FE06C081E0C81AD10879
:105E4000E10880E8F80AC882D982EA82FB82C701A9
:105E5000B6019F77DF91CF91FF90EF90DF90CF90C9
:105E6000BF90AF909F908F9008958F929F92AF9226
:105E7000BF92CF92DF92EF92FF9260910D017091ED
:105E80000E0180910F01909110016115710581053E
:105E9000910521F464E279ED8BE597E02DE133EF94
:105EA00041E050E00E94383149015A019B01AC01A8
:105EB000A7EAB1E40E9457316B017C01ACEEB4EF6C
:105EC000A50194010E946531C60ED71EE81EF91E79
:105ED000F7FE06C081E0C81AD108E10880E8F80A98
:105EE000C0920D01D0920E01E0920F01F0921001CC
:105EF000C701B6019F77FF90EF90DF90CF90BF90E2
:105F0000AF909F908F90089560930D0170930E0154
:105F100080930F01909310010895FB01DC0105901F
:105F20000D920020E1F70895FC0105900020E9F7AB
:105F3000809590958E0F9F1F0895BB274A3031F4AE
:105F4000992322F4BDE2909581959F4F0C94DA2F0E
:105F5000BB272A3051F4992342F4BDE290958095F5
:105F6000709561957F4F8F4F9F4F0C94B82FBB2733
:105F7000FA01A62F6217710581059105330B30FBDD
:105F800066F0AA27660F771F881F991FAA1FA217FE
:105F900010F0A21B63953850A9F7A05DAA3308F052
:105FA000A95DA19336F7B111B1931082CA010C9487
:105FB000F32FBB27FB015527AA27880F991FAA1F7C
:105FC000A41710F0A41B83955051B9F7A05DAA3314
:105FD00008F0A95DA193009779F7B111B1931192DF
:105FE000CB010C94F32FDC01FC01672F7191772317
:105FF000E1F7329704C07C916D9370836291AE1784
:10600000BF07C8F30895E89409C097FB3EF4909544
:106010008095709561957F4F8F4F9F4F9923A9F081
:10602000F92F96E9BB279395F69587957795679510
:10603000B795F111F8CFFAF4BB0F11F460FF1BC054
:106040006F5F7F4F8F4F9F4F16C0882311F096E9E7
:1060500011C0772321F09EE8872F762F05C0662395
:1060600071F096E8862F70E060E02AF09A95660F4E
:10607000771F881FDAF7880F9695879597F9089507
:10608000990F0008550FAA0BE0E8FEEF1616170649
:10609000E807F907C0F012161306E407F50798F0B1
:1060A000621B730B840B950B39F40A2661F0232BCA
:1060B000242B252B21F408950A2609F4A140A69546
:1060C0008FEF811D811D08950E9477300C94E83078
:1060D0000E94DA3038F00E94E13020F0952311F070
:1060E0000C94D1300C94D73011240C941C310E94A4
:1060F000F93070F3959FC1F3950F50E0551F629FE3
:10610000F001729FBB27F00DB11D639FAA27F00D10
:10611000B11DAA1F649F6627B00DA11D661F829F37
:106120002227B00DA11D621F739FB00DA11D621F1C
:10613000839FA00D611D221F749F3327A00D611D39
:10614000231F849F600D211D822F762F6A2F11241B
:106150009F5750409AF0F1F088234AF0EE0FFF1F4E
:10616000BB1F661F771F881F91505040A9F79E3FA5
:10617000510580F00C94D1300C941C315F3FE4F356
:10618000983ED4F3869577956795B795F795E795FB
:106190009F5FC1F7FE2B880F911D9695879597F904
:1061A000089597F99F6780E870E060E008959FEF99
:1061B00080EC089500240A9416161706180609069E
:1061C000089500240A94121613061406050608956D
:1061D000092E0394000C11F4882352F0BB0F40F4F5
:1061E000BF2B11F460FF04C06F5F7F4F8F4F9F4F35
:1061F000089557FD9058440F551F59F05F3F71F0B7
:106200004795880F97FB991F61F09F3F79F087951D
:106210000895121613061406551FF2CF4695F1DFA6
:1062200008C0161617061806991FF1CF8695710536
:10623000610508940895E894BB2766277727CB016A
:1062400097F90895F999FECF92BD81BDF89A9927E3
:1062500080B50895262FF999FECF1FBA92BD81BD52
:1062600020BD0FB6F894FA9AF99A0FBE01960895D8
:10627000052E97FB1EF400940E944F3157FD07D066
:106280000E94A13107FC03D04EF40C944F3150957D
:106290004095309521953F4F4F4F5F4F0895909512
:1062A0008095709561957F4F8F4F9F4F08950E9405
:1062B000C331A59F900DB49F900DA49F800D911D9B
:1062C00011240895B7FF0C9457310E945731821B57
:1062D000930B08952F923F924F925F926F927F920D
:1062E0008F929F92AF92BF92CF92DF92EF92FF92E6
:1062F0000F931F93CF93DF93CDB7DEB7CA1BDB0B92
:106300000FB6F894DEBF0FBECDBF09942A88398836
:1063100048885F846E847D848C849B84AA84B9843D
:10632000C884DF80EE80FD800C811B81AA81B98149
:10633000CE0FD11D0FB6F894DEBF0FBECDBFED015D
:106340000895A1E21A2EAA1BBB1BFD010DC0AA1FB6
:10635000BB1FEE1FFF1FA217B307E407F50720F0CE
:10636000A21BB30BE40BF50B661F771F881F991F49
:106370001A9469F760957095809590959B01AC0192
:10638000BD01CF010895A29FB001B39FC001A39F9B
:10639000700D811D1124911DB29F700D811D11245E
:1063A000911D08955058BB27AA270E94EA310C94EA
:1063B000E8300E94DA3038F00E94E13020F039F401
:1063C0009F3F19F426F40C94D7300EF4E095E7FBC8
:1063D0000C94D130E92F0E94F93058F3BA176207B4
:1063E00073078407950720F079F4A6F50C941B3108
:1063F0000EF4E0950B2EBA2FA02D0B01B9019001E0
:106400000C01CA01A0011124FF27591B99F0593F23
:1064100050F4503E68F11A16F040A22F232F342F6B
:106420004427585FF3CF469537952795A795F040B9
:106430005395C9F77EF41F16BA0B620B730B840BCE
:10644000BAF09150A1F0FF0FBB1F661F771F881F86
:10645000C2F70EC0BA0F621F731F841F48F48795DE
:1064600077956795B795F7959E3F08F0B0CF9395D0
:10647000880F08F09927EE0F9795879508950E9449
:1064800053320C94E8300E94E13058F00E94DA3028
:1064900040F029F45F3F29F00C94D13051110C9455
:1064A0001C310C94D7300E94F93068F39923B1F372
:1064B000552391F3951B550BBB27AA27621773072A
:1064C000840738F09F5F5F4F220F331F441FAA1FBE
:1064D000A9F335D00E2E3AF0E0E832D0915050407A
:1064E000E695001CCAF72BD0FE2F29D0660F771F28
:1064F000881FBB1F261737074807AB07B0E809F00E
:10650000BB0B802DBF01FF2793585F4F3AF09E3F92
:10651000510578F00C94D1300C941C315F3FE4F3BA
:10652000983ED4F3869577956795B795F7959F5FD5
:10653000C9F7880F911D9695879597F90895E1E021
:10654000660F771F881FBB1F621773078407BA0780
:1065500020F0621B730B840BBA0BEE1F88F7E095DB
:1065600008950E94B8326894B1110C941C310895BA
:106570000E94013188F09F5798F0B92F9927B751A1
:10658000B0F0E1F0660F771F881F991F1AF0BA95D7
:10659000C9F714C0B13091F00E941B31B1E00895E9
:1065A0000C941B31672F782F8827B85F39F0B93FDB
:1065B000CCF3869577956795B395D9F73EF490958A
:1065C0008095709561957F4F8F4F9F4F08950E94E2
:1065D000273390F09F3748F4911116F00C941C313A
:1065E00060E070E080E89FEB089526F41B16611DC3
:1065F000711D811D0C94FE320C941933882371F4A3
:10660000772321F09850872B762F07C0662311F44B
:1066100099270DC09051862B70E060E02AF09A9582
:10662000660F771F881FDAF7880F9695879597F979
:1066300008959F3F31F0915020F4879577956795A5
:10664000B795880F911D9695879597F908950E94A3
:106650000131A0F0BEE7B91788F4BB279F3860F47A
:106660001616B11D672F782F8827985FF7CF86956C
:1066700077956795B11D93959639C8F308950E9453
:10668000403008F48FEF089519F416F40C94D730C5
:106690000C9419330E940131B8F39923C9F3B6F36E
:1066A0009F57550B87FF0E948A330024A0E640EADB
:1066B000900180585695979528F4805C660F771F57
:1066C000881F20F026173707480730F4621B730B2A
:1066D000840B202931294A2BA6951794079420254D
:1066E00031254A2758F7660F771F881F20F0261795
:1066F0003707480730F4620B730B840B200D311DF4
:10670000411DA09581F7B901842F9158880F969566
:106710008795089591505040660F771F881FD2F7D4
:106720000895DB018F939F930E945731BF91AF91E2
:10673000A29F800D911DA39F900DB29F900D1124DB
:106740000895EE0FFF1F0590F491E02D09940F932B
:106750001F93CF93DF938230910510F482E090E095
:10676000E091AA07F091AB0730E020E0B0E0A0E0B4
:10677000309799F42115310509F44AC0281B390BCB
:1067800024303105D8F58A819B816115710589F125
:10679000FB0193838283FE0111C0408151810281FC
:1067A000138148175907E0F04817590799F41097D3
:1067B00061F012960C93129713961C933296CF01A8
:1067C000DF91CF911F910F9108950093AA07109325
:1067D000AB07F4CF2115310551F04217530738F0BC
:1067E000A901DB019A01BD01DF01F801C1CFEF0171
:1067F000F9CF9093AB078093AA07CDCFFE01E20FAC
:10680000F31F819391932250310939832883D7CF85
:106810002091A8073091A907232B41F4209113015F
:10682000309114013093A9072093A80720911101FA
:10683000309112012115310541F42DB73EB7409139
:10684000150150911601241B350BE091A807F0911A
:10685000A907E217F307A0F42E1B3F0B28173907EF
:1068600078F0AC014E5F5F4F2417350748F04E0FAC
:106870005F1F5093A9074093A807819391939FCFDF
:10688000F0E0E0E09CCFCF93DF930097E9F0FC01CC
:10689000329713821282A091AA07B091AB07ED0143
:1068A00030E020E01097A1F420813181820F931F06
:1068B0002091A8073091A9072817390709F061C06E
:1068C000F093A907E093A807DF91CF910895EA011B
:1068D000CE17DF07E8F54A815B819E01411551051E
:1068E000B1F7E901FB83EA8349915991C40FD51FA0
:1068F000EC17FD0761F4808191810296840F951F4A
:10690000E90199838883828193819B838A83F0E064
:10691000E0E012968D919C9113970097B9F52D9117
:106920003C911197CD010296820F931F2091A807E9
:106930003091A9072817390739F6309751F5109289
:10694000AB071092AA07B093A907A093A807BCCFE2
:10695000D383C28340815181840F951FC817D90703
:1069600061F44E5F5F4F88819981480F591F5183B1
:1069700040838A819B81938382832115310509F0AD
:10698000B0CFF093AB07E093AA079ECFFD01DC01E7
:10699000C0CF13821282D7CFB0E0A0E0E2EDF4E3E3
:1069A0000C946C318C01009751F4CB010E94A733F9
:1069B0008C01C801CDB7DEB7E0E10C948831FC0151
:1069C000E60FF71F9C0122503109E217F30708F484
:1069D0009DC0D901CD91DC911197C617D70798F0CA
:1069E000C530D10530F3CE0104978617970708F319
:1069F000C61BD70B2297C193D1936D937C93CF0184
:106A00000E944334D6CF5B01AC1ABD0A4C018C0EF8
:106A10009D1EA091AA07B091AB07512C412CF12CDF
:106A2000E12C109731F58091A8079091A90788155E
:106A3000990509F05CC04616570608F058C08091C9
:106A4000110190911201009741F48DB79EB74091CA
:106A5000150150911601841B950BE817F90708F0F2
:106A600055C0F093A907E093A807F90171836083EB
:106A7000A0CF8D919C91119712966C9012971396BE
:106A80007C901397A815B90559F56C0142E0C40E26
:106A9000D11CCA14DB0420F1AC014A195B09DA01EC
:106AA0001296159780F06282738251834083D901D8
:106AB0006D937C93E114F10471F0D7011396FC936C
:106AC000EE93129776CF22968C0F9D1FF90191833A
:106AD0008083F301EFCFF093AB07E093AA0769CF70
:106AE0004816590608F42C017D01D3019ACFCB0139
:106AF0000E94A7337C01009749F0AE01B8010E94C3
:106B00008935C8010E944334870153CF10E000E06B
:106B100050CFFB01DC0102C001900D92415050406A
:106B2000D8F70895FB01DC0101900D920020E1F7F8
:106B3000089517E0CCEAD7E004C0FE010E94A1331B
:0C6B40002196CD3AD107C9F7F894FFCF99
:106B4C0010FFFFFFFF00E10000000000000100004B
:106B5C00000000AC07800000C18081000000000034
:106B6C000000F00B5B0D110C060C570C150C330CC4
:106B7C00000000004B12C50E7813E00D0000000061
:106B8C00FD11C50E7813E00D00000000C510C50EF8
:106B9C007813E00D596F752068616C6C7563696EC4
:106BAC00617465206F6E207468650077696C64652C
:106BBC0073742074726970206F6620796F7572001F
:106BCC006C6966652C207374756D626C65206F6ED4
:106BDC00746F2074686500737562776179207472C4
:106BEC0061636B732C20616E642067657400637243
:106BFC0065616D6564206279206120747261696ED3
:106C0C002E002020204A75737420736179206E6FDA
:106C1C000020202020746F2064727567732E002072
:106C2C002047616D65206F76657221002020596FB9
:106C3C0075722073636F72653A200020206F757433
:106C4C00206F66203130302E006F6E20612064651D
:106C5C006164206475646520696E007468652073D6
:106C6C00756277617921212100546865206D61720C
:106C7C006B657420686173006265656E20666C6F6D
:106C8C006F6465642077697468006368656170205F
:106C9C00686F6D656D6164650061636964212121B4
:026CAC002100C5
:00000001FF
